:1000000000400020714C0000B14C0000B34C0000D7
:1000100000000000000000000000000000000000E0
:10002000000000000000000000000000B54C0000CF
:100030000000000000000000B74C0000B94C0000B8
:10004000BB4C0000BB4C0000E1550000BB4C000065
:10005000BB4C000000000000BB4C0000BB4C00008B
:10006000BB4C0000894E0000BB4C0000BB4C0000A4
:10007000BB4C0000BB4C0000BB4C0000BB4C000064
:10008000BB4C00004D4D0000BB4C0000BB4C0000C1
:10009000BB4C0000BB4C0000BB4C0000BB4C000044
:1000A000BB4C0000BB4C0000000000000000000042
:1000B0000000000000000000000000000000000040
:1000C000054B0648033310B51B1A062B03D9044B06
:1000D000002B00D0984710BD64010020640100206F
:1000E000000000000648074910B5091A8910CB0F17
:1000F0005918491003D0044B002B00D0984710BD6D
:1001000064010020640100200000000010B5074CCD
:100110002378002B09D1FFF7D3FF054B002B02D02A
:10012000044800E000BF0123237010BD64010020DB
:1001300000000000E08C0000094B10B5002B03D03C
:100140000849094800E000BF08480368002B02D1B5
:10015000FFF7C8FF10BD064B002BF9D09847F7E713
:100160000000000068010020E08C00006001002019
:1001700000000000164B002B00D1144B9D4640227E
:1001800092029A1A924600218B460F461348144A4F
:10019000121A08F080FA0F4B002B00D098470E4B34
:1001A000002B00D098470020002104000D000D48CE
:1001B000002802D00C4800E000BF08F029FA200017
:1001C000290005F037FA08F00DFAC04600000800D3
:1001D000004000200000000000000000640100203A
:1001E000780A0020000000000000000082B00190AA
:1001F000019B002B17D0019B013B01930B4B1A0075
:10020000013B002AF4D0C046C046C046C046C046A6
:10021000C046C046C046C046C046C046C046C046AE
:10022000C046C046EBE702B07047C046E703000097
:10023000F7B507000800019208F040F802000B0033
:100240000020274906F012FE08F006F90021061CDE
:1002500005F00CFC041E41D12249301C05F0D6FFEC
:10026000FC21890505F0D2FF06F06AFA0500019825
:1002700006F088FA311C05F0FFFD06F061FA060071
:10028000A6422BDD0121380004F062FE002D0ED0C5
:1002900028000138C046C046C046C046C046C046D9
:1002A000C046C046C046C046C046C046F1D1002147
:1002B000380004F04DFE002D0ED028000138C04655
:1002C000C046C046C046C046C046C046C046C046FE
:1002D000C046C046C046F1D10134D1E7F7BDC046A3
:1002E00000408F4000007A4410B5024802F0B0FF91
:1002F00010BDC046D406002010B5024802F0FEFF33
:1003000010BDC046D406002010B5044C200003F0F8
:1003100094F8200002F0F2FF10BDC046D406002081
:10032000F8B5160012021A431C000B0407000D005A
:100330001A4381B2064803F047F8032F06D803207A
:100340007843044B1E54181845708470F8BDC0469D
:10035000D406002082010020F0B50400002589B0F9
:1003600001910292039305AE019B605D5B5D029972
:10037000181A05F045FAAF000135B851032DF3D135
:100380000027029A7BB2013A934223DA00252378B0
:100390003268D318237072686378D3186370B268B8
:1003A000A378D318A370EDB2A37828006278013542
:1003B0002178FFF7B5FFEBB2DDB2042BF3D1FFF7E5
:1003C0009BFF0299039805F01BFA013704F0B0FC7B
:1003D000FFB2D6E70024019B019A0199E4B29B7811
:1003E0002000527801340978FFF79AFFE3B2DCB2BB
:1003F000042BF0D1FFF780FF0299039805F000FA73
:1004000004F096FC09B0F0BD10B52A4B2A4A002131
:10041000092813D805F056F91211110F0D0B090711
:10042000120504210AE0FC2108E0F82106E0F4218D
:1004300004E0F02102E0EC2100E0D8219950A12154
:100440000720C90058500638083158501B4C1C4929
:10045000184A5C501B4C04315C501B4C1B495C50CF
:100460001B4C04315C5000211A4C195104341851B2
:1004700019481950A3211948C90058500220184999
:100480005850585803231840022804D11549164BD8
:10049000D150164908E051580B40012B06D1FF21DD
:1004A000114BD1500821FF31043BD1500320FFF7FD
:1004B0009DFE10BD001000400C050000E7C2C3C443
:1004C00024050000C8C7C6C5E7E7E7E71C0500002C
:1004D000C2C2C2002C05000014050000050504017D
:1004E00034050000FFFF00003C0500002110010062
:1004F0000022094B10B55A6080220121D2051160FB
:100500005A68002AFCD0054B1868FFF77DFF044BA2
:10051000044A0549D15010BDFC000040F0060020FF
:1005200004050000001000405C02002030B5134CB0
:10053000134DA17000212D78E2702371114A124BE6
:1005400025706070D450114B5960013111605A68A8
:10055000002AFCD001210B4A916000210B4A116155
:100560001A69002AFCD00021084A5161054A01316C
:1005700011615A69002AFCD030BDC0465C020020DF
:10058000B90600200010004004050000FC100040E7
:1005900030B50024114A124B1249D150124B5C6005
:1005A000013454605C68002CFCD000250E4C2561A1
:1005B0000A4C0135A5601C69002CFCD08024074D35
:1005C000E4002C59012C00D1087800215961013137
:1005D00011615A69002AFCD030BDC04600100040AD
:1005E000040500005C020020FC10004000231900FC
:1005F000024A99540133102BFBD17047BC010020F3
:1006000000230549FF201A025242800212185A5054
:100610000433802BF6D17047DC01002080220023B8
:10062000FF200349D200585401339342FBD1704755
:1006300064020020134A30B50123904220D882057D
:100640001ED1114A926F90421AD3022180250F4B7E
:100650000F4AED00995080245959E4000029FAD03E
:10066000A1210A4DC900685019590029FCD0002069
:10067000064988508021C9005A58002AFCD000231E
:10068000180030BDFFFF0300DC01002000E0014046
:1006900004050000174BF0B5070001209F4227D842
:1006A000BB0525D18B0723D1134B9B6F9F421FD3D3
:1006B000124C134B26001851053CFF3C18590028DA
:1006C000FCD08020C000002484468020C000A242CC
:1006D00008D9A50048597851604618580028FBD021
:1006E0000134F2E700229A511A58002AFCD0002067
:1006F000F0BDC046FFFF0300DC0100200405000040
:1007000000E0014070B500241F4D0121605D04F040
:1007100001FC605D002104F01BFC605D00210134E0
:1007200004F0F8FB032CEFD10024184E0121A05D4A
:1007300004F0F0FBA05D0021013404F009FC032C5F
:10074000F3D100242600A85D04F010FB0136241824
:10075000052004F0EDFA032EF5D10D4B1A689442F2
:1007600004DDF422FF32944200DC1C60094B1A685D
:10077000944200DA1C600321200005F041F8064B8A
:100780001870200070BDC046880000207C0000204A
:10079000CC01002084000020B401002010B500240A
:1007A0000F4B0121E05C013404F0D2FB092CF7D19E
:1007B00000240C4B0021E05C013404F0C9FB032C45
:1007C000F7D1094A531D0A3211000022581F027046
:1007D0001A705A719A72DA7301339942F6D110BDC8
:1007E000880000207C0000208E01002010B500242D
:1007F000094B0121E05C013404F08CFB092CF7D19A
:100800000024064B0121E05C013404F083FB032C3F
:10081000F7D1FFF7C3FF10BD880000207C00002047
:10082000F0B587B0059004F051FA039000251E4BF7
:100830006C0001341C19052300266B431B4AD31896
:100840000493049B9B5D002B1DD0631E1B7800212D
:100850000193019A164B985C04F07AFB2378154FAC
:100860000121F85C029304F073FB012004F060FAAC
:100870000F4B019A0121985C04F06AFB029B002156
:10088000F85C04F065FB01360A34052ED9D1013538
:10089000052DCCD104F01AFA039BC01A059B98428F
:1008A000C4D307B0F0BDC046498900008E010020C6
:1008B000880000207C000020F0B55A4B85B0051E52
:1008C00001919D4208DC584CA04203DB00900028B7
:1008D00004DA0400634200E0544B00930A210098BC
:1008E00005F074F8009803910A2104F089FF0A21A9
:1008F00005F06CF84E4A531D0A32100000225E1FAC
:1009000032701A705A719A72DA7301338342F6D1D7
:10091000019B002B10D12B000933122B0FD8039B06
:10092000444A5B00D2180292434A0120D318039331
:100930003F4B00229C464EE0019B012B1CD83D4BB7
:1009400049005B180293012000230521029A5943B4
:10095000D75C374A511800220424A41AA4463C004C
:1009600066463441044200D088540132052AF3D14E
:100970000133022BD3D0E8E7019B022BCFD12E4BC2
:1009800049005B180293012000230521029A594374
:10099000D75C274A511800220424A41AA4463C001C
:1009A00066463441044200D088540132052AF3D10E
:1009B0000133022BB3D0E8E7019C002C12D1029C3A
:1009C000A75C0F41074200D0187001330139F3D200
:1009D0000132022A08D0052353430F336344042114
:1009E0006646E9E7039CEBE72B006333C62B04D88C
:1009F000002D14DA0123B37211E06421009804F091
:100A0000FFFE0E4B0122195C002308001841104222
:100A100001D0F01A82730133052BF6D1E8E705B057
:100A2000F0BDC046E60300000DFEFFFFE703000037
:100A30008E010020AE89000090890000A48900008A
:100A4000F8B5150006000F001C00FFF7CFFE2800C8
:100A500007F034FC02000B0000200A4902F0F8FC09
:100A600032003B0006F026FE07F0F2FB2900FFF7FC
:100A700023FF20000A38FFF7D3FE0A2004F058F9BC
:100A8000F8BDC0460000244080221A4B1A491B685A
:100A9000D20070B59818CC1A1A78E25401330A00C3
:100AA0008342F9D10C78154B15481C604B88154DC5
:100AB000036089882960168913490E70134EB3426A
:100AC00003D100232B6003600B70114BD188114DB3
:100AD000197000239C420CD9190008314900565C5A
:100AE00051185800497846550133281841709BB277
:100AF000F0E770BDDC01002064020020D006002079
:100B0000F8060020B8010020F4060020FFFF0000D6
:100B10007000002009070020164B70B51868164BAE
:100B2000164C1B68164D6380164B20701B68A38003
:100B3000154B1B78E380154B1B785BB22381002398
:100B400098420CD91A0059004E5D083269185200BB
:100B50004978A6540133A21851709BB2F0E70C4DAE
:100B60002868FFF767FD8022286852002100FFF700
:100B700091FD70BDD0060020F80600206402002020
:100B800009070020B801002070000020F4060020B2
:100B9000DC010020F0B5444C8FB01922210007A8D9
:100BA00007F070FD21001022193103A807F06AFD3B
:100BB000FFF76AFF3D4A3E4D13780192FF2B00D1AB
:100BC00000233C4C2B60200004F016FA3A49200028
:100BD00004F008FA0A222968200004F064FA0023CD
:100BE0000093334B009A1B689A425AD21300019A21
:100BF00008335B00D55CD31814222E4C5E7802AB10
:100C00009B18595D200004F0F1F92B000A3B2700E6
:100C1000012B02D9EB1F012B03D8380004F0ECF9AB
:100C20003BE0062D12D12549200004F0DBF90F230B
:100C300003AA3340D15C200004F0D8F92049F30620
:100C400002D4B30629D51F4920001AE02B000C3B23
:100C5000012B19D820001C4904F0C4F907243300E3
:100C600001222341134205D008230932191B1148E0
:100C700004F043FA013CF2D214490D2D00D114497D
:100C8000380004F0C1F908E00C49200004F0AAF98A
:100C90000A223100200004F0FCF9009B01339BB2D2
:100CA0009EE70FB0F0BDC04620890000640200201E
:100CB000D0060020040A0020D28900002A8A000001
:100CC000E0890000E3890000E6890000EB8900006C
:100CD000EA89000070B5084D084C2B789B00185924
:100CE000FFF7A8FC80222B7852009B00044918597A
:100CF000FFF7D0FC70BDC04670000020DC01002072
:100D000064020020F7B50090019103F0DFFF1A4D57
:100D100007002B7800201E2B2CD8FE23174CFF3306
:100D200022889A4208D9FFF7D5FF2B7801332B7020
:100D300000232380FFF772FC114B1868114B381AFF
:100D4000984202D96422104B1A800F4B25881988CB
:100D500004F0CCFC6A460D4E6B00985312786B1C65
:100D60005B00F254F6186B461B7902357370044B26
:100D700025801F60FEBDC04670000020C406002014
:100D8000C8060020FFFF00000400002064020020CD
:100D9000F0B585B0039300900191029203F096FFA5
:100DA0001D4D07002B7800201E2B32D8FE231B4C34
:100DB0005B0022889A4208D9FFF78CFF2B78013319
:100DC0002B7000232380FFF729FC154B1868154B67
:100DD000381A984202D96422134B1A80124B258884
:100DE000198804F083FC6A46104E6B009853127801
:100DF0006B1C5B00F254F6186B461B79033573705D
:100E00006B461B7A2580B3706B461B7BF370044BDB
:100E10001F6005B0F0BDC04670000020C406002071
:100E2000C8060020FFFF000004000020640200202C
:100E300037B50021051C04F03DFE094C002803D005
:100E40000849200004F0CEF8281C07F0B1FA0B0086
:100E5000032102000091200004F0FCF93EBDC046D1
:100E6000040A00202A8A000070B50849051E084CB3
:100E7000092D02D9632803D80649200004F0B2F8EE
:100E800029000A22200004F000F970BD298A000020
:100E9000040A00202A8A0000F0B5724C87B02000B6
:100EA00004F0AAF87049200004F0AEF86F4B1F1D43
:100EB0007833059300230393019380223B68D2008B
:100EC00099186B4AD21A1878D05401339942FAD142
:100ED0000025674B6A00D25A02920299654A9142F4
:100EE00004D10235644B9D42F3D9B3E00299039AD1
:100EF0008C46013203926C1C019A5A4E6400624483
:100F00001B5D019203990A223000049304F0B1F8AA
:100F10005A49300004F066F8049B30009A00584BA0
:100F2000D15804F05FF85549300004F05BF8554B98
:100F30001B88012B02D10A22019903E064210A22B5
:100F4000019B5943300004F094F84C49300004F000
:100F500049F8049B581E0C285FD8454B04F0B2FB9F
:100F600007070707102907073047070707001C195D
:100F70006078FFF779FF41493A4804F033F84CE0D4
:100F80000326023C3A4B1B19985707F097F9FE23AA
:100F900000229B0506F08EFB07F05EFAFFF748FF84
:100FA000013636492F4804F01DF8062EEAD10335E4
:100FB0003DE01C196078C043C0B2FFF755FF27E041
:100FC0000326023C2A4B1B19985707F077F9002299
:100FD0002D4B06F06FFB07F03FFAFFF729FF0136B4
:100FE0002A49204803F0FEFF062EEBD1DFE701205F
:100FF0001C19205607F062F90022254B06F05AFB17
:101000000022244B05F006FC07F026FAFFF710FF3C
:101010001A49144803F0E6FF04E0FB22049B053B59
:101020001342C4D01C490F4803F0DCFF0235154BB6
:101030000C4C1B88012B02D10A22029903E0642187
:101040000A22029B5943200004F013F8200003F009
:10105000D3FF47E7059B04379F4200D02DE70020D0
:1010600007B0F0BD040A0020EE890000DC0100207A
:1010700064020020FFFF0000FF010000258A00003D
:1010800008000020040000200000903F1F8A00009C
:101090000000E03F00003940238A0000F8B504005A
:1010A0002B4E300003F0A8FF601E0C284FD8294CAF
:1010B00004F008FB0707070709210707273E070772
:1010C000070020781AE00025605707F0F7F8FE23A4
:1010D00000229B0506F0EEFA07F0BEF9FFF7A8FE26
:1010E0006F1C022D33D01C49300003F07BFF3D1EE6
:1010F000032DE9D12BE02078C043C0B2FFF7B4FE46
:1011000025E00025605707F0D9F80022134B06F0C0
:10111000D1FA07F0A1F9FFF78BFE6F1C022D16D054
:101120000D49300003F05EFF3D1E032DEAD10EE0B5
:10113000207807F0C3F80022094B06F0BBFA002222
:10114000084B05F067FB07F087F9FFF771FEF8BD64
:10115000040A0020B4010020258A00000000903F0E
:101160000000E03F0000394010B5002911D1002AED
:1011700011D010000138C046C046C046C046C04627
:10118000C046C046C046C046C046C046C046F1D173
:1011900001E0FFF74DF810BD012170B5080003F024
:1011A000D7FE0A200138C046C046C046C046C046E9
:1011B000C046C046C046C046C046C046C046F1D143
:1011C0000021012003F0C4FE022003F0D7FE002816
:1011D000FAD003F093FD00240500022003F0CEFEB8
:1011E000012803D103F08AFD0400F6E7601B07F035
:1011F000A7F80B4B002205F039FE07F02DF909493D
:10120000041C04F04DFC0300FF20002B02D1201C25
:1012100005F096FA044B18700A23584370BDC04677
:1012200000004D4000007F43B401002000238020D7
:101230001A0010B5054980005A54CC180233627068
:101240008342F9D10022024B1A6010BD0907002029
:10125000D006002000230E4A70B513600D4A0E48D8
:1012600013600E4A0E4913601A001A505A50043384
:10127000282BFAD1002301251A000A4E0A4C0B49EB
:1012800098009A551D55013342500A2BF7D170BD75
:10129000AC010020A8010020640600208C0600207C
:1012A00090060020D10100203C09002014090020F4
:1012B00010B5FA24FFF7CEFF0122084B64001A7024
:1012C000210031320020FEF7B3FF322003F030FD61
:1012D000322221000020FEF7ABFF10BD810100206B
:1012E00010B5FA210024084B3222890020001C701E
:1012F000FEF79EFF322003F01BFDFA213222490047
:101300002000FEF795FF10BD8101002010B50021DF
:101310000D2003F0FFFD00210E2003F0FBFD002156
:10132000052003F0F7FD00210B2003F0F3FD012160
:10133000082003F0EFFD01210C2003F0EBFDFFF787
:1013400089FFFFF7CDFF0121080003F0E3FD002135
:10135000022003F0DFFD00210E2003F0DBFD002161
:101360000D2003F0D7FD0021012003F0F1FD10BD99
:101370000F4B10B51B780400002B18D00D2808D88F
:101380000C4BC340DB0704D50B4B1978FFF7BAFCB5
:101390000AE0FB22631F134209D1074920008B7822
:1013A0004A780978FFF7F4FC2000FFF777FE10BDBC
:1013B000B8060020DE3D0000B401002070B5040036
:1013C0000D00FFF713FA6000012D00D12843002320
:1013D00001240A4D0022204202D0D11A69188C74CF
:1013E000053A110040080F31F5D10133032BF1D13B
:1013F000FA204000FFF714FA70BDC0468E010020AD
:1014000070B50500082401262800013C2041304029
:1014100009D0FA21322289000020FEF709FF962028
:1014200003F086FC04E0FA21C8228900FEF700FFE1
:10143000962003F07DFC002CE6D170BD10B50400B1
:10144000000AC0B2FFF7DCFFE0B2FFF7D9FF10BD22
:1014500070B50500042401262800013C20413040DD
:1014600009D0FA21322289000020FEF7E1FE962001
:1014700003F05EFC04E0FA21C8228900FEF7D8FEE2
:10148000642003F055FC002CE6D170BDC31710B5E5
:10149000C4185C40002802DA0F20FFF7D9FF632C44
:1014A0000CDDFA212000890004F090FA0800642184
:1014B00004F0A6F9C0B2FFF7CBFF01E0092C0ADD6A
:1014C0006421200004F082FA08000A2104F098F94F
:1014D000C0B2FFF7BDFF20000A2104F077FAC8B2BE
:1014E000FFF7B6FF642003F023FC10BD194B10B5C5
:1014F000041E9C4213DD184904F082F906F0DEFE5A
:10150000FA2300229B00FFF79BFA6421200004F0DD
:1015100077F9642104F05AFA6431080004E0632882
:101520000FDD642104F06CF906F0C8FEFA230022F6
:101530009B00FFF785FA6421200004F047FA64312C
:10154000080006F0BBFEFA2300229B00FFF778FAA2
:1015500010BDC0460F2700001027000010B50E2058
:1015600003F00CFD43425841C0B210BD10B50D2030
:1015700003F004FD43425841C0B210BD00230100F6
:101580001A0010B50E4C002918DB4800005D063823
:1015900005280FD804F096F8030E07090D0701334C
:1015A000012B07D108E0013B04E00132012A01D1FF
:1015B00004E0013A0139E6E7180000E0002010BD20
:1015C0000907002010B5064C52230F2204212000E9
:1015D00001F0E4FE034A0449200006F0E7FF10BDD5
:1015E000D4060020000000203532000070B5164CF3
:1015F0001021200001F0A2FD0021200001F0C9FC13
:101600000021200001F0C5FC104D20002978403158
:10161000C9B201F0BEFC200001F0FAFD200010214B
:1016200001F08CFD0221200001F0B3FC002120001C
:1016300001F0AFFC297820004031C9B201F0A9FCCB
:10164000200001F0E5FD70BD48090020F4060020EF
:1016500070B5164C1021200001F070FD0021200013
:1016600001F097FC0121200001F093FC104D2000B7
:1016700029784031C9B201F08CFC200001F0C8FD8E
:101680002000102101F05AFD0221200001F081FC10
:101690000121200001F07DFC297820004031C9B2F1
:1016A00001F077FC200001F0B3FD70BD4809002077
:1016B000F406002070B5164C1021200001F03EFD0C
:1016C0000021200001F065FC0121200001F061FCF7
:1016D000104D200029784031C9B201F05AFC200099
:1016E00001F096FD2000102101F028FD02212000CC
:1016F00001F04FFC0021200001F04BFC2978200074
:101700004031C9B201F045FC200001F081FD70BDFF
:1017100048090020F406002070B5164C1021200066
:1017200001F00CFD0021200001F033FC002120001D
:1017300001F02FFC104D200029784031C9B201F092
:1017400028FC200001F064FD2000102101F0F6FCCF
:101750000221200001F01DFC0121200001F019FCF4
:10176000297820004031C9B201F013FC200001F0BB
:101770004FFD70BD48090020F406002010B5144C40
:101780001021200001F0DAFC0021200001F001FC12
:101790000021200001F0FDFB0021200001F0F9FBF9
:1017A000200001F035FD2000102101F0C7FC0221CE
:1017B000200001F0EEFB0021200001F0EAFB0021F7
:1017C000200001F0E6FB200001F022FD10BDC04624
:1017D0004809002010B5041CFFF708FF0649201C2B
:1017E00004F014FD04F09CF903F0A2FAFFF7C6FF21
:1017F000642003F09DFA10BD0000C84210B5041C1F
:10180000FFF726FF0649201C04F000FD04F088F9CC
:1018100003F08EFAFFF7B2FF642003F089FA10BDDF
:101820000000C84210B5041CFFF744FF0649201C05
:1018300004F0ECFC04F074F903F07AFAFFF79EFF71
:10184000642003F075FA10BD0000C84210B5041CF6
:10185000FFF762FF0649201C04F0D8FC04F060F991
:1018600003F066FAFFF78AFF642003F061FA10BD07
:101870000000C84270B506000D00084C1021200081
:1018800001F05CFCF1B2200001F083FBE9B2200022
:1018900001F07FFB200001F0BBFC70BD4809002077
:1018A00010B50F4C0821200001F048FC0721200052
:1018B00001F06FFB0021200001F04CFC0123082106
:1018C0001A00200001F0D0FB200001F05DFBC2B245
:1018D0000023FF2A02D0034BC0B21B5C180010BDCE
:1018E00048090020C289000010B50400FFF7D8FFA6
:1018F000002803D1200003F01BFAF7E710BD70B5F4
:1019000001253220FFF7F0FFFA210400642289004C
:101910000020FEF78DFC2300313BDBB2082B05D8FD
:101920000A206843303C0419E0B205E0302C02D1B3
:1019300001350A2DE5D1002070BD000000231A00FA
:10194000F0B585B001AC1A550133092BFBD1012646
:101950003220FFF7C9FF0500313DEDB2082D07D851
:10196000FA21642289000020FEF762FC6655EFE749
:101970003028EDD1FA21002064228900FEF758FCBE
:101980000023032718009C463D000D499A1D8A1824
:1019900000215D4365196E5C012E02D11670304343
:1019A00001E0664616704000013180B2053203291D
:1019B000F1D10133032BE7D1400805B0F0BDC0469B
:1019C0008E01002070B5060003F080F905000400C8
:1019D000FFF766FF002809D1641BB44206D23230FB
:1019E00003F0A6F903F072F90400F1E770BD0000FE
:1019F00070B50600154C1E21200001F09FFB310040
:101A0000200001F0C6FA200001F002FC022001389B
:101A1000C046C046C046C046C046C046C046C04696
:101A2000C046C046C046C046F1D101221E2120005A
:101A300001F07FFB200001F0A2FA002804D0200072
:101A400001F0A2FAC5B2F5E7280070BD48090020F0
:101A500010B54F20FFF7CCFF40284BD1264C1E215C
:101A6000200001F06BFB6021200001F092FA0021C0
:101A7000200001F08EFA200001F0CAFB1E21200098
:101A800001F05CFB6221200001F083FA01212000BB
:101A900001F07FFA200001F0BBFB1921200001F0CA
:101AA0004DFB2321200001F074FA8021200001F079
:101AB00070FA200001F0ACFB1921200001F03EFB80
:101AC0002021200001F065FA5721200001F061FA81
:101AD000200001F09DFB1921200001F02FFB1F21A8
:101AE000200001F056FAC021200001F052FA200037
:101AF00001F08EFB10BDC04648090020F8B50F006C
:101B0000164CC5B22900200001F018FBF9B22000E4
:101B100001F03FFA200001F07BFB05200138C046B0
:101B2000C046C046C046C046C046C046C046C04685
:101B3000C046C046C046F1D101222900200001F074
:101B4000F8FA200001F01BFA002804D0200001F070
:101B50001BFA0600F5E73000F8BDC0464809002032
:101B600070B505001600FFF7C9FF04000520013815
:101B7000C046C046C046C046C046C046C046C04635
:101B8000C046C046C046C046F1D131002800FFF72C
:101B9000B5FFE4B20002204300B270BDF0B5692287
:101BA00085B068211E20FFF7DBFF6B226A2107004A
:101BB0001E20FFF7D5FF6D2206006C211E20FFF7C7
:101BC000CFFF584D2B689F4200DD2F60564C236895
:101BD0009F4200DA2760554B1A68964200DD1E606E
:101BE000534B1A68964200DA1E60524B1A689042B4
:101BF00000DD1860504B1A68904200DA18602B68BC
:101C000022689918CB0F59184C4B49101960474B53
:101C10001B680193464B1B680293019B1A00029BB1
:101C20009C466244D30F9A1853100293029A444B75
:101C30001A60404B1B6801933F4B1B680393019B49
:101C40001A00039B9C4662441300D20F94463D4AFF
:101C500063445B1013607A1A0192029AC31AB21A93
:101C600018000392029306F029FB06000F0001986A
:101C700006F024FB32003B0001F0E6FB019BDE177F
:101C80009A19039B7240DE179B197340D318029A6E
:101C9000D617921972409B18FA22D20093420BDC9D
:101CA0000022294B05F006FD284A294B05F0DEF8F5
:101CB00006F0D2FB041C13E00023224A1360204AE2
:101CC00013601E4A1360234B1A4A2B601360174A95
:101CD0001360214B184A236000241360144A1360D8
:101CE000201C06F065FBFA2300225B00FEF7A8FE2D
:101CF0000320019A194BD7170740BF18039ABF104A
:101D0000D6170640B618029AB610D2171040029A9B
:101D10001F708018801098705E70201C04F010FDF9
:101D200005B0F0BD78000020800000206C0000208D
:101D3000940000207400002068000020FC060020B1
:101D40000007002004070020008066407A008BFC1A
:101D5000FA2109400A00FFFFF6FF0000B40100204D
:101D6000F7B5292228211920FFF7FAFE2B220400BB
:101D70002A211920FFF7F4FE2D2207002C2119201B
:101D8000FFF7EEFE384B22121A703A125A70021206
:101D900006009A70200006F091FA0022334B05F0FD
:101DA00089FC040038000D0006F088FA00222F4B51
:101DB00005F080FC00900191300006F07FFA0022CF
:101DC0002A4B05F077FC220006000F002B002000B4
:101DD000290005F06FFC009A019B04000D00100023
:101DE000190005F067FC02000B002000290004F038
:101DF00011FD320004000D003B003000390005F0F9
:101E000059FC02000B002000290004F003FD01F042
:101E1000F7FC174A04000D0000980199154B03F0D8
:101E200005FE012600281DD10022134B20002900A9
:101E300005F0BAFE0022002304000D0003F0F6FDB9
:101E40000E4A002805D00E4B2000290003F0EEFDBD
:101E500004E00C4B2000290003F0D4FD002800D141
:101E6000061CF6B23000FEBDB40100200000103F99
:101E700039B4C876BE9FE6BF0000F03F9A999999A1
:101E80009999C93F9999C9BF70B5052407211920AF
:101E9000FFF734FE0C211920FFF730FE2000013837
:101EA000C046C046C046C046C046C046C046C04602
:101EB000C046C046C046C046F1D10D211920FFF7EB
:101EC0001DFE030020000138C046C046C046C04683
:101ED000C046C046C046C046C046C046C046C046D2
:101EE000F1D10E4A58B2137004F04CFCFC21890564
:101EF00004F08CF90A4903F049FE051C04F020FCAB
:101F00000400281C06F054FAFA2301229B00FEF775
:101F100097FD2000FFF7BAFA200070BDB401002041
:101F20000000C84110B5041E0E2C69D803F0CAFB8E
:101F30000D0D161668680808222D363C41415200E6
:101F40000520062C3DD006303BE0634263410E2065
:101F5000C01A03F013F82B4B187039E0FFF71CF987
:101F600063230138032C01D02C23FF3383428041AB
:101F7000404246E0FEF7C6FB234B02001B680120EF
:101F80000E3B9A423DDB00203BE0FFF707FE0300DB
:101F90001E2200200F339A42404132E0FFF7E0FE5C
:101FA0000138434258412CE0FFF76EFF08231538F3
:101FB000DCE70C3C601E84410021200002F0AAFFF7
:101FC000200002F0DBFFC3B25A4253410D4A1370A6
:101FD000C0B216E00021022002F09CFF022002F0B5
:101FE000C5FE084B8408E0B2187006F0A9F9FA2380
:101FF00000225B00FEF724FD60B2C043C00F00E08A
:10200000012010BDB4010020CC01002010B5022039
:10201000FFF788FF431E9841C0B210BD10B50320E2
:10202000FFF780FF431E9841C0B210BD10B50620D7
:10203000FFF778FF431E9841C0B210BD10B50720CE
:10204000FFF770FF431E9841C0B210BD10B50C20C1
:10205000FFF768FF431E9841C0B210BD10B50D20B8
:10206000FFF760FF431E9841C0B210BD10B50E20AF
:10207000FFF758FF0138431E9841C0B210BD10B59C
:102080000820FFF74FFF0138431E9841C0B210BD32
:1020900010B50920FFF746FF0138431E9841C0B232
:1020A00010BD10B50A20FFF73DFF0138431E9841CF
:1020B000C0B210BD10B50B20FFF734FF0138431E2E
:1020C0009841C0B210BD0000824BF7B51B780500E7
:1020D0000F00002B00D19CE07F4B1B78002B53D1CD
:1020E000FEF756FA7D4BC0B21A787F23824201D1A7
:1020F0007B4B5B7859B27B4C002905DA7F22134079
:1021000000220F2B03D903E00F2B01D80122E25448
:10211000754B1B78002B13D0714A744B9078187054
:10212000D078587012799A706B1E012B02D90A3B35
:10213000012B01D8002903DA39002800FFF718F92C
:10214000635D002B1BD13B00103B5A425A41D3B276
:10215000BEE0FFF76BFF061E00D0AAE0802000263D
:102160002843A37862782178FEF7E0F96B461B7963
:10217000012B4AD90B3D022D47D9002EE3D0103F49
:102180007B1E9F41FBB2A3E0431E0193574C0C2BD7
:1021900033D8180003F08CFADD13070A28250D1038
:1021A0002B2E161B2000FFF739FF87E0FFF72EFFCD
:1021B00084E0FFF7DBF981E0FFF7D0F97EE0FFF77D
:1021C0003DFFC8E7FFF742FF061EC7D017E0FFF745
:1021D00045FF061E63D1C1E7FFF748FF061E63D126
:1021E000BCE7FFF74CFF69E0FFF752FF66E0FFF73F
:1021F00058FF63E0FFF75EFF60E00126B1E70B20C8
:10220000A37862782178FEF791F9142002F090FD0E
:10221000B3E701380D285BD803F054FA15180F12F4
:102220002724070A2A2D1B1E2130FFF79FF901E002
:10223000FFF794F9002886D0A1E7FFF7EFFEF9E752
:10224000FFF7E4FEF6E7FFF7F1FEF3E7FFF7F6FE30
:10225000F0E7FFF7FBFEEDE7FFF700FFEAE7FFF728
:1022600005FFE7E7FFF70BFFE4E7FFF711FFE1E703
:10227000FFF717FFDEE7FFF71DFFDBE71C4B1A68D0
:10228000102901D1013200E0013A1A60186806F005
:1022900015F8C8230022FEF7D3FB012318E0A3782A
:1022A000627821780C20AEE7A378627821780D203F
:1022B000A9E7A378627821782800A4E7002800D154
:1022C0004CE7A378627821782800FEF72FF956E7CB
:1022D0001800FEBDEC06002010090020B906002001
:1022E0005C020020BC010020B8060020B4010020E0
:1022F000B0010020F8B5A94AA94D12682B689A428E
:1023000019D2FEF7EDFFFDF7FFFF0021082002F0D4
:102310001FFE00210C2002F01BFEA24B1B78002B9D
:1023200001D0FDF7F1FFA04B1B78002B00D112E28A
:10233000FEF7D0FC0FE29D4A5B009E5CD3185C78F0
:10234000221E09D1731E042B02D9143B032B03D880
:102350000A2003F061F9C2B2954B954F1B68002B20
:102360001CDD9448591E8446405C002816D0062E79
:1023700008D0082E0FD0072E00D1BFE10B2E00D0C1
:10238000E6E108E08A495A1C0A6001226146CA5403
:102390002B689B18DEE1864A1160D9E1701E172870
:1023A00000D9D2E103F098F918001E0024002A0099
:1023B00030007401AA01B8014B016001BF013B006C
:1023C0003900D101D101D101D101D101D101D10116
:1023D00040004C005A001201100004F0D3F9FFF73E
:1023E000F9F9B2E1100004F0CDF9FFF707FAACE11A
:1023F000100004F0C7F9FFF715FAA6E1100004F089
:10240000C1F9FFF723FAA0E16B4B5200D15AFA222F
:1024100000205200FEF7A8FE97E1012100E0002114
:102420002000FEF7CBFF90E1200005F047FF0022DF
:10243000624B05F03FF905F00BFF010014200AE0A4
:10244000200005F03BFF00225C4B05F033F905F05E
:10245000FFFE01001520FFF70DFA9AE0012C05D1CF
:102460002100082002F074FD210004E00021082072
:1024700002F06EFD00210C2002F06AFD494B1B7832
:10248000002B00D161E14E4E4E48337803707178D5
:102490004170B2788270072C2BD18B4203D19342CA
:1024A00001D15B0834E05C18802C03D1802912D163
:1024B000602306E08C18802C08D1802A0ED00B00F7
:1024C000203B737013002033B3700BE09C18802CFA
:1024D00008D1802B02D1203B337033E0203AB27018
:1024E00020333370FA2308225B003100FDF734FFFC
:1024F0002BE1092C34D18B4211D193420FD1002B07
:1025000001D1013304E05AB2002A04DB5B00DBB2E4
:102510003370B37018E0FF23B3707370E1E75C1899
:10252000802C04D1802B18D020397170D8E78C18FA
:10253000802C0BD1802902D160227270D0E7130069
:10254000203BB3700B0020337370CBE79C18802CBA
:10255000C8D1802A01D16023F3E7203B3370B1E773
:1025600003235C43184B1A5D1C1963783270737037
:10257000A378B3700023DCB27278B378317820008E
:10258000FDF7CEFE631CDAB2D3B2042AF3D1FDF715
:10259000B3FEFA20400002F0CBFBD6E0D0060020CC
:1025A000AC01002061020020B806002009070020CD
:1025B0008C060020D10100207C89000000003440FE
:1025C000ED060020CC060020480000200A21200053
:1025D00003F08CF8C0B205F071FE02000B00002081
:1025E0005D4900F035FF06000F0020000A2103F0CE
:1025F00003F9C8B205F062FE32003B0005F05AF85C
:1026000005F026FE0400002C12DD200005F056FE29
:10261000524B0022FEF714FA0A20FFF7D3F92A28BA
:1026200001D0232802D1FEF75BFE94E0013CEAE7EB
:102630006423002200210020FEF702FA85E0484AC8
:10264000484913689B00002C02D1FF20C85000E0CD
:10265000CC50136844492C68980001334450092B2E
:1026600000DD0923136070E03D4C3E482368591E8D
:102670008A001358FF2B07D0012B01D1216064E0A1
:10268000012B62DD013B1350374BD3582B605CE0CC
:10269000364A2868990001338850092B00DD092348
:1026A0003B6026000F231E409C4321003000FFF7B3
:1026B0000BFD3B682E4A013B002804D00021D15479
:1026C0002C4AD15403E00121D1542A4AD054731E1C
:1026D000012B02D90A3B012B03D8102C01D1002871
:1026E00033D0254B1B78002B2FD0244B1B78002B8D
:1026F0002BD121003000FEF73BFE26E01C4A013BB7
:10270000D15C1C48002903D0C15C00291DD101E027
:102710000121C154D15418E000221549013BCA548B
:102720001449CA5408E01248013BC15C114A00290F
:1027300004D00021C154D1543B6006E0D1540B4A6F
:1027400099008A583B602A6005E00A2002F0F0FAFE
:102750002B6801332B60F8BD00002440DE0300002D
:10276000A801002090060020640600201409002023
:10277000D10100203C090020B8060020EC06002012
:10278000E12110B54902154802F0B0FD01210020F9
:1027900002F0C0FBFEF7BAFDFDF732FFFEF774F959
:1027A0000F4800F02FFCFFF753F90E4B1A68FF2A71
:1027B00001D100221A601A680B4B1A6000220B4BE1
:1027C0001A600B4B1B78934203D0FDF78DFDFDF78C
:1027D0009BFD084800F03CFD10BDC046040A0020E7
:1027E00048090020D0060020BC060020B0010020CF
:1027F00061020020D406002070B5CA4C2678012E54
:1028000038D1FFF74DF8C84B18702A2814D1FEF7BD
:1028100067FD0022C54B1A60C54B1B78934204D05C
:10282000FEF758FAC34802F067FDC34B1B78002B34
:102830001ED0FDF769FD1BE0232819D1BF4D2B7871
:10284000002B04D102F042FA02F0E0FE2E700025C7
:10285000FEF746FDBA4B1D60FEF7E8FC0122B34BC4
:102860001D60B84B1A70B24B1B78AB42DDD0D7E776
:10287000FFF740FD2678002E00D067E3FFF710F841
:10288000A94D2870002800D160E32A282BD1AC4C38
:10289000AD4B22681868AB49AC4D904202D1087824
:1028A00001280DD11A6000230B70A9492A600B681A
:1028B00001330B60A7490B689B180B60FEF72CF9DE
:1028C000FEF7F6FC23682B60FDF7A8FE02F0FEF988
:1028D000A14B002118600123A04A1370A04A118067
:1028E000A04A138032E3A04C23281DD1FA21642290
:1028F00089003000FDF79CFCFEF798FC924B2660A7
:102900001A68002A02D001218E4A117000221A6032
:10291000864B8B491A60884B0A601B78934200D122
:1029200014E3FDF7F1FC11E3302800D04AE1844EB6
:102930003368002B00D045E12068002800D041E139
:10294000FA2164228900FDF773FC3220FEF7CCFFE8
:1029500028703038052800D927E102F0BDFE0600B6
:102960000A006C00A500250013010C20FEF748FDAD
:102970001BE1C8204000FFF725F8754C287000289F
:1029800002D0312807D1734C2068FEF757FD20682C
:10299000FEF7ACFD09E1302800D006E100236D4AC6
:1029A00013606B4A136043E0FA216422890000201F
:1029B000FDF73EFC3220FEF797FFFA2128706422D3
:1029C00089000020FDF734FCFEF75EF82B78312BF0
:1029D00008D1664B1A78023AD2B251B22F310BDAD3
:1029E000D02209E0372B0FD1604B1A780232D2B2D5
:1029F00051B22F2900DD302200201A70185605F040
:102A00005DFCC823002211E0342B07D10020574B76
:102A1000185605F053FCFA235B00F3E7302B07D17F
:102A20000022524B00201A700021C823FEF708F83C
:102A3000FEF772F8B9E0FA21642289000020FDF760
:102A4000F7FB3B4B1C78002C02D0FEF725FAACE0DC
:102A5000474B1B78002B3DD00121464A13784B4051
:102A600013702BD0FA21322289002000FDF7E0FB01
:102A7000FA2322005B0040490020FDF7E1FFFA2025
:102A8000FEF7A0FF3D4B2870002801D1186008E038
:102A90003038186005F012FCFA2322005B00FDF7C5
:102AA000CFFFFDF725FD80E00122314C2378534014
:102AB0002370FDF79BFD2378002B0ED1FA21C8224D
:102AC00089000020FDF7B4FBFA2300225B00002000
:102AD000002168E0FEF75EF867E0FDF709FD0024DD
:102AE000FA21244B3222890020001C70FDF7A0FB44
:102AF000FA2322005B0020490020FDF7A1FFFA2005
:102B0000FEF760FF1E4B2870A04201D118704CE008
:102B10003038C0B2187005F013FCFA2322005B00B5
:102B200041E0C0468101002080010020B00100206A
:102B3000B8060020040A00206102002008070020D7
:102B4000BC060020D00100200C090020D006002087
:102B5000F8060020B8010020C80600207000002000
:102B6000C406002004000020C0060020F406002057
:102B7000EC060020100900200000F03FF0060020C5
:102B8000B90600200121B44A13784B40137095D048
:102B9000FA21322289000020FDF74AFBFA230022A5
:102BA0000020AE495B00FDF74BFFFDF76DFFAC4B1E
:102BB0001A68FF2A01D100221A601B68A94A3360F3
:102BC0001360C3E12068002800D0A6E0FA21642247
:102BD0008900FDF72DFB0123287823602338212865
:102BE00000D9B3E102F078FD9200B201B201B20166
:102BF000B201B201B2018501B201B201B201B2016A
:102C0000B2016600220027002E00440049004E0059
:102C100053005B006000B201B201B201B201B20127
:102C2000B201B201730078007D008D008E4B092146
:102C30001B685B0003E001218B4B1B685B008B4A28
:102C4000995483E1884E35682800FEF797FC874A3F
:102C50006B00002804D10A21D154D318587004E025
:102C60000B21D154D31800225A700135356040E150
:102C70007D4B03211B685B00E1E77B4B05211B6853
:102C80005B00DCE7784B04211B685B00D7E706217B
:102C9000754B764A1B685B00995402232AE1724BFC
:102CA00002211B685B00CAE76F487049036808256A
:102CB0005A0004E007256C486C4903685A005554D3
:102CC0008A18002101335170036021603EE1664B98
:102CD00015211B685B00B2E7634B16211B685B0084
:102CE000ADE71721604B614A1B68614C5B0099544A
:102CF0002378002B00D029E1FDF7F6FA0123237099
:102D000024E1594B18211B685B0098E70025564BBE
:102D10001D60FEF78BFA256018E1012854D1FA21D5
:102D2000002064228900FDF783FA002328782360BD
:102D300030384D4D092800D905E12B684B4C5B001C
:102D400002F0C0FC2005080B0E1114171A1DE41820
:102D5000012337E0E418022334E0E418032331E0D0
:102D6000E41804232EE0E41805232BE0E4180623DE
:102D700028E0E418072325E0E418082322E0E418FB
:102D800009231FE0E25C052A11D1FEF7D7FD0028D8
:102D900011D04210C30703D52B680D215B0002E060
:102DA0000C212B685B00E154E4186270CBE0182A18
:102DB00006D1FEF7A4FD2B685B00E4186070C2E04A
:102DC000E41800236370BEE0022800D094E0FA21EA
:102DD000002064228900FDF72BFA03232878236062
:102DE0003038142800D97EE002F06CFC590B12191F
:102DF00020272E44524B7D7D7D7D7D7D7D60676EDD
:102E00007500194B194A1B685B00D318032268E050
:102E1000154B164A1B685B00D318052261E0124B64
:102E2000124A1B685B00D31804225AE00E4B0F4A6B
:102E30001B685B00D318012253E00B4B0B4A1B6845
:102E40005B00D31806224CE0074B084A1B685B0066
:102E5000D318022245E0C046B80600200000F03F2B
:102E6000D00600200C090020BC0600200907002025
:102E700061020020364B374A1B685B00D3180722DB
:102E80002FE0334B334A1B685B00D318082228E03D
:102E90002F4B304A1B685B00D318092221E02C4BD2
:102EA0002C4A1B685B00D3180A221AE0284B294AD7
:102EB0001B685B00D3180B2213E0254B254A1B68C7
:102EC0005B00D3180C220CE0214B224A1B685B00EC
:102ED000D3180D2205E01E4B1E4A1B685B00D31859
:102EE0000E225A7032E0FA21642249000020FDF7D8
:102EF0009FF90023236029E0032827D1FA21002627
:102F0000642289000020FDF793F92B782660104D8C
:102F1000322B08D0382B0FD12B680E4A5B00D31808
:102F20005A78202105E010212B680A4A5B00D3184B
:102F30005A780A435A7006E0FA21642249003000A8
:102F4000FDF776F926602B6801332B6070BDC04613
:102F5000BC06002009070020F8B505000E00170088
:102F60000024BC4208D02B68315D1B6828009847BC
:102F7000002801D00134F4E72000F8BD704710B5F7
:102F80001C3002F098F910BD10B51C3002F085F924
:102F900010BD70B5437E0D00002B05D064300400D9
:102FA00002F098F9002801D0002004E02000290058
:102FB00002F064F9012070BD10B51C3002F081F9F7
:102FC00010BD0000F7B50193FA23002504009B0013
:102FD00083600B4B4560083303601C300F00160004
:102FE00002F041F92000643002F03DF96B461B7994
:102FF000276166756576A5762000A375FEBDC0467F
:10300000588A0000012330B5A024C375837D12497E
:103010009B005A58437DC1329B005B580F4DC13312
:10302000FF32FF33E40592009B0015511D51CC2463
:1030300003690B4A64049C500524243A9C50827D09
:1030400092005458A122D2009C50427D92005158C7
:10305000044A995030BDC046788A00000C06000032
:10306000240500000C050000F7B5050000200C0049
:10307000019382425CD0161E402E00D940262F00BC
:103080001C37380002F005F9B1222B69D2008021EB
:103090009C50012289005A50A97E002901D11A6250
:1030A0001A600024731E2A69A34206D1019B002BDB
:1030B00003D0802302219B00D1500123136213000F
:1030C000FC33D968002902D1996A0029F9D0996A9C
:1030D00000290AD1D960A323DB00D1583800C9B236
:1030E000013402F0CBF8A642DCD8019A2B69002A01
:1030F00004D11A00FC32916A00290AD00121002271
:10310000AA7659611900FC3188680028FCD08A60D1
:1031100007E00121A976D961D16C0029FCD00021FA
:10312000D164FC339A6A002A01D000229A62E0B28C
:10313000FEBD10B50123FFF797FF10BD0300AC33B0
:1031400010B504001970643002F0A3F8012363760F
:1031500010BD0000F8B500220D0001004276AC3130
:10316000036904000878B121C90058508021890002
:103170005A5001321A629A6026006436300002F01A
:103180009AF800280ED03000276902F086F81E4B0E
:10319000F8502369FC331A6A002A0CD19A6A002A73
:1031A000F9D008E02369002D0AD11A00FC32916A97
:1031B000002905D10EE09A6A002AF3D11A62DBE7F2
:1031C00001225A611A00FC3291680029FCD00021CA
:1031D000916006E00121D961D16C0029FCD0002169
:1031E000D1641A000020FC32916A81420BD0074959
:1031F00090625A5802305A50824204D0043A5342E4
:1032000053410230C01AF8BD1C050000C404000080
:1032100010B50121FFF79EFF10BD000010B513236C
:10322000142202490248FFF7CDFE10BD00400040C5
:103230004809002010B50400C06805F019FA0623FB
:10324000E05E002802DB002101F064FE200010BDDA
:1032500010B504000623C05E002809DB012101F03F
:1032600059FE0623E05E002101F072FE012000E01D
:103270000020607010BD70B50500C0680E0005F03C
:10328000F7F9EB7C2C7C1C1B63425C4104231C1B68
:103290007443A4B2AC80200005F0E0F9E860002897
:1032A00005D02200002105F0F6F96E8001E0A8802B
:1032B000688070BDC37C027C70B59A1A5442544138
:1032C000E2B203248B110D118E10264023402540BD
:1032D0000C4046748474FF2600248E426441C16809
:1032E000C37405740470002907D05B1B5C425C4109
:1032F000944202D04188FFF7BEFF70BDF8B5C368A5
:103300000400002B2BD001F0F9FC6369984200D235
:1033100060616369C01A2C23FF339842F3D972B6F7
:103320000621635E0E499B005B580121A2889940EB
:103330000C48E36808E001602F4200D141607F083B
:1033400007D10133013A05D38027C04641601D787B
:10335000F1E7FBE7416062B601F0D0FC6061F8BDC7
:10336000788A00000805005070B5437804000D000D
:10337000002B06D00623C05E002802DB002101F0EE
:10338000C9FD6378E580002B07D00121280001F0FA
:10339000C1FD0021280001F0DBFD70BD70B51500F6
:1033A000002204000E0042700272C26042611900E5
:1033B000FFF780FF31002000FFF75DFF29002000AC
:1033C000FFF7D2FF200070BD4388F7B58B4233D999
:1033D000037A150C140A002B04D1E4B2EDB2019467
:1033E000D6B20AE0FF26344035405C4316405D43C8
:1033F0005E43240A2D0A0194360A077CB446C67C33
:103400003C1EC768B44203D1032359437F180AE026
:1034100089007F18120EBE19002B01D1D3B201E032
:1034200053431B0A33706A46037C1279FD54437C74
:10343000FA546246837CFA54F7BD10B500218288A5
:10344000C06805F028F910BD10B500F035FA10BDC0
:10345000F0B5454657464E46E0B48EB016001F0004
:1034600004000D0000F0E4FA0A000100CE4B0291C6
:10347000039298461B78009101925BB2013305D00C
:103480003000390001F0ACFA002807D1009801990A
:103490000EB01CBC90469946A246F0BD2000290003
:1034A00001F09EFA00228246002837D10023300026
:1034B000390002F0A1FA0028E8D004AB99460123B4
:1034C0004A460493B94B494653604B4652461A62EA
:1034D00000229C60DD601E615F61B54B8A61CB613B
:1034E000414609780092019349B2481CCED0022986
:1034F000CCD0484601F0A2FA002800D1C2E04B46E9
:103500001B6A002B04D005F067F84B461B6A03606A
:103510004B46DC699B6900930194B7E700232000C8
:10352000290002F069FA002823D00022002330008D
:10353000390002F061FA824600282FD004AB994688
:1035400001234A460493994B9460D560536000234D
:103550000024136200239361D46143461B781661F3
:1035600057615BB2002BC4D00023914C00930194AF
:103570008CE70298039901F029FA8246002800D1CD
:1035800085E0029803990022002302F035FA002812
:1035900036D1029B039C0093019477E730003900F9
:1035A00001F014FA002800D170E700220023300057
:1035B000390002F027FA002800D167E704AB9946EA
:1035C00001234A460493794B53604B4652469C6014
:1035D000DD601A621E615F6143461B78002B00D0DC
:1035E0007EE04A46002300249361D461484601F0FE
:1035F00025FA00287CD04B461B6A002B88D082E736
:103600002000290001F0E2F9029A039B0092019345
:10361000002800D13AE73000390001F0D7F9029ACA
:10362000039B00920193002800D12FE704AB994639
:1036300004234A4604935D4B9460D5605360002395
:103640000024136200239361D46143461B78166102
:1036500057615BB2022B04D0484601F0EFF9002815
:10366000C9D104F0B9FF22230360C4E7002300227C
:103670001900100003F0FAFB4B469861D961022C47
:1036800000D036E704F0A8FF2123036037E72000CD
:10369000290001F09BF9002800D172E730003900C1
:1036A00001F094F9002800D16BE70298039901F02A
:1036B00097F904AB994600281FD101234A46049389
:1036C0003A4B9460D560536043461C781062166193
:1036D0005761002CCAD1002300249361D46108E70C
:1036E00000204A4633499061D161022B00D07DE72A
:1036F00004F072FF212303607DE703234A4604930D
:103700002A4B53604B4652469C60DD601A621E6134
:103710005F6143461B785BB2002B18D1E02249461B
:10372000254B12068A61CB6120000022002329006C
:1037300002F068F900281DD1484601F07FF9002801
:1037400000D0DCE604F048FF22230360D7E6002225
:1037500049461A4B20008A61CB61002200232900D0
:1037600002F050F900282FD143461B785BB2022BA0
:10377000E2D1E7E70022124B3000390003F09AFF54
:1037800004000D0001F062F902000B002000290086
:1037900002F032F90028E7D1E0224946094B12062F
:1037A0008A61CB61E0E7C04698000020FC8A0000F7
:1037B0000000F03F0000F0FFFFFFEF470000F07F48
:1037C0000000E03FFFFFEFC700220B4B3000390045
:1037D00003F070FF04000D0001F038F902000B0047
:1037E0002000290002F008F90028BDD10022494636
:1037F000024B8A61CB61B7E70000E03F0000F0FFB9
:10380000F0B5474680B48CB004000D0000F046FED1
:10381000274B060098461B780F005BB201330DD092
:103820002000290001F0DCF8002807D00022002346
:103830002000290002F0E6F8002805D13000390008
:103840000CB004BC9046F0BD01230293194B0694C2
:103850000795039300230A934346049405951C7827
:10386000002C0FD1002300240893099402A801F032
:10387000E5F8002810D00A9B0193002B11D1089E77
:10388000099FDBE7002200231000190003F0EEFA85
:1038900008900991022CE9D104F09EFE21230360D7
:1038A000E9E704F099FE0A9B01930360E7E7C0464D
:1038B00098000020008B0000F8B515004F464646E2
:1038C0005A001C006B42C0B42B434B4F5208DB0F15
:1038D00088461343BB423AD84B005B0899464E4694
:1038E00043420343DB0F3343BB4230D8434BE3181F
:1038F0002B4343D00226A3171E40CB0F1E434B463B
:1039000003432ED013002B4332D0BA4241D0B945E5
:103910002ED04B469A1A12153C2A32DC002C55DB6D
:103920002A00230003F0A2FA01F04CF800F0ACFEEC
:10393000012E46D0022E39D0002E0ED0304A314B07
:1039400004F032F9304A314B04F02EF905E0020060
:103950000B002800210002F05DFF0CBC9046994648
:10396000F8BD022E10D0032EF7D127482849F4E7DE
:1039700043462548002B0ADB2649EEE700F084FE8B
:10398000EBE721482349D3E71F482049E5E72249CF
:10399000E3E791451FD0022EF6D0032EE5D000209C
:1039A0000021012ED9D180210906D6E7144A154BF2
:1039B00004F0FAF802000B001348144904F0F4F87C
:1039C000CBE7802424060B191900C6E73C32A7DA9E
:1039D00000200021ACE7022E06D0032E09D00A48B1
:1039E000012E04D00D49B8E70D480E49B5E70E4940
:1039F000B3E70B480D49B0E70000F07F000010C0AE
:103A0000075C143326A6A13C182D4454FB21094021
:103A1000FB2109C0FB21F93FFB21F9BFFB21E93F55
:103A2000D221337F7CD90240FB21E9BF7CD902C07F
:103A3000F0B556464D4644465F46F0B41C001300B0
:103A4000670091B07F080093019406000D00804646
:103A50008946A2463B4332D06E4B6C0064089C42C0
:103A600029DC26D09F4226DC6A4B9F4200D189E0A8
:103A700000239B464B46002B00DA87E0002A2FD11B
:103A8000644B9F4200D19FE0634B9F425DD08023F7
:103A9000DB059A4501D100F0C1FB604B9A451FD16F
:103AA0004B46002B1CDB3000290000F0F7FC060021
:103AB00007E000280DD05A4BE01830430BD1002608
:103AC0005549300011B03CBC90469946A246AB46E1
:103AD000F0BDA742C8DD534800F0B2FF0600F0E792
:103AE0003000290000F06EFF4346002B1DD0EB0F85
:103AF000013B98465B464246134379D04A4B9F426E
:103B000000DC9FE0494B9F4201DC00F0CEFB484BBC
:103B10009C4279DD5346002B79DD464A464B100026
:103B2000190003F0C7FD0600CBE7002C04D03A4A89
:103B3000AB009B089342DAD15346002B00DAADE389
:103B40004B46002B0DDB0600BBE753462900002B3C
:103B5000B7DA32002B0000202F4903F087F9060066
:103B6000AFE72F4B9C465B4664441C4301D100F0F9
:103B70002BFC5B460600012BA3D180231B069C4631
:103B800061449EE7002A00D172E794E72B4B9F42E5
:103B90002BDC274B9F4200DC70E729493B158C4604
:103BA0006344142B01DC00F0F2FB3421CB1A0099A2
:103BB000D94008009840824200D05FE701231940B5
:103BC00001335B1A9B4659E7154BE018064300D1B9
:103BD00075E7174B9C4200DC51E35346002B16DB84
:103BE000009B019C1E0021006BE702239B4645E7DA
:103BF00032002B003000290003F0D6FF02000B003A
:103C000003F034F906005CE75346002B85DB002601
:103C1000002156E70000F07F0000F03F0000E03F89
:103C2000000010C0048B00000000E0410000F043E1
:103C3000FFFFEF3F9C7500883CE4377EFFFF3F436A
:103C400001FCFFFFE84B00229C4206DC0022E74B10
:103C500003F030FD35220C005242E54D2315AC46F1
:103C6000634499462403E34DE34B240B91442543DD
:103C70009C4209DDE14B9C4200DCA9E301239C4608
:103C8000DF4BE1449C466544002300240022089356
:103C900009940C930D940024D64B06920793069A30
:103CA000079B29000A900B9103F07EFF069A079B61
:103CB00006000F000A980B9902F0ACFD02000B0001
:103CC0000020CC4903F0D2F80A00010013000E9145
:103CD0000F9202003900300003F0ECFC0A000100F2
:103CE0008020049105921300002280210003844665
:103CF00002920393002289056D100D4365442B1930
:103D00000298039914001D0003F0D4FC02000B007C
:103D10003000390003F048FF069A079B06000F00A9
:103D20002000290003F040FF02000B000A980B99C5
:103D300003F03AFF029A039B03F0BCFC02000B0065
:103D40003000390003F030FF0E9A0F9B03F0B2FCF5
:103D5000049D059E069007912A003300280031003B
:103D600003F0A8FC06000F00A64AA74B03F0A2FC34
:103D7000A64AA74B02F04EFD32003B0003F09AFC2E
:103D8000A44AA54B02F046FD32003B0003F092FC32
:103D9000A24AA34B02F03EFD32003B0003F08AFC36
:103DA000A04AA14B02F036FD32003B0003F082FC3A
:103DB0009E4A9F4B02F02EFD320004000D003B0096
:103DC0003000390003F076FC02000B0020002900CF
:103DD00003F070FC029E039F04000D0004980599F7
:103DE00032003B0002F016FD069A079B03F062FCCE
:103DF00022002B0002F00EFD32000A900B913B00D6
:103E0000300039000296039703F054FC0022894BDE
:103E100004000D0002F0FEFC0A9A0B9B02F0FAFC73
:103E200000260F0032000B000298039903F042FCB9
:103E30000022029003917F4B3000390003F0B4FE62
:103E400022002B0003F0B0FE02000B000A980B9931
:103E500003F0AAFE049A059B03F02CFC3200040038
:103E60000D00069807993B0003F024FC02000B00AC
:103E70002000290002F0CEFC04000D0002000B001F
:103E80000298039902F0C6FC0026E0226A4B120653
:103E900030000F0003F00EFC029A039B0490059182
:103EA0003000390003F080FE02000B0020002900E2
:103EB00003F07AFE614A604B03F0FCFB604A0400A9
:103EC0000D00604B3000390003F0F4FB02000B00E2
:103ED0002000290002F09EFC0C9A0D9B02F09AFC37
:103EE000060048460F0004F0E9F904000D000498AC
:103EF000059932003B0002F08DFC089A099B02F004
:103F000089FC22002B0002F085FC002022002B00FF
:103F10000290039103F048FE089A099B03F044FEC7
:103F2000049A059B03F040FE02000B0030003900AC
:103F300003F03AFE049005915B464246013B134371
:103F400000D197E100232B4C069307940098019928
:103F500000260B0032000F0003F026FE029A039B9E
:103F600003F0A8FB009A019B04000D00049805993A
:103F700003F0A0FB02000B002000290002F04AFC25
:103F800004000D00029803993B003200049405954B
:103F900003F090FB009001910B000200290020002B
:103FA00002F038FC284B81460F1E8A469F4200DCF7
:103FB0003CE1264BCB18034300D0DBE10498059984
:103FC000234A244B02F026FC009A019B04000D00BA
:103FD0004846390003F0E8FD02000B0020002900EC
:103FE00001F024FD3E0037E0FFFF0F0000004043DA
:103FF00001FCFFFF0000F03F8E98030079B60B0034
:104000000000F0FFEF4E454A287ECA3F65DBC993AA
:104010004A86CD3F01411DA96074D13F4D268F5185
:104020005555D53FFFAB6FDBB66DDB3F0333333305
:104030003333E33F0000084009C7EE3FFD033ADC9D
:10404000F5015B14E02F3EBEFFFF8F40000070BF04
:10405000FE822B654715973C002800D08AE180221C
:10406000E74B52039C461300361566443341E5493D
:10407000DB195E001C001B038C461B0B1343142230
:10408000760DE14F66443741961B334198465346BF
:10409000BC4300202100002B00DAA9E102000B0044
:1040A0000098019903F080FD0B000090019102003F
:1040B0000498059902F0AEFB43461B059946002083
:1040C0000022D24B06000F0003F0F4FA009A019B85
:1040D000029003913000390003F066FD02000B00EE
:1040E0000498059903F060FDC94ACA4B03F0E2FA4F
:1040F000C94A04000D00C94B3000390003F0DAFA58
:1041000002000B002000290002F084FB04000D00D7
:1041100002000B000298039902F07CFB029A039BB9
:1041200006000F0003F040FD02000B0020002900F4
:1041300003F03AFD3200009001913B00300039005D
:1041400003F0B8FA04000D00B54AB64B03F0B2FA1A
:10415000B54AB64B03F028FD22002B0003F0AAFA63
:10416000B34AB44B02F056FB22002B0003F0A2FA34
:10417000B14AB24B03F018FD22002B0003F09AFA6B
:10418000AF4AB04B02F046FB22002B0003F092FA3C
:1041900002000B003000390003F006FD04000D00A2
:1041A00002000B003000390003F084FA80230290F3
:1041B00003910022DB052000290003F0F5FC02003A
:1041C0000B000298039902F051FE009A019B040033
:1041D0000D003000390003F06DFA009A019B02F0E7
:1041E00019FB02000B002000290003F0DDFC320067
:1041F0003B0003F0D9FC02000B000020924903F0C1
:10420000D3FC4B465B181A15002A00DCF4E01900B9
:10421000069A079B03F04EFA060052E43200300083
:104220002B00290003F046FA06004AE4874B4E00B3
:1042300076089E4200DCBFE0854BCB1803430CD1CF
:10424000009A019B03F0B0FC02000B000498059952
:1042500001F0E2FB002800D101E7069807997D4AAA
:104260007D4B03F027FA7B4A7B4B03F023FA0600D1
:10427000FFF727FC0023794C0693079466E6534624
:10428000002B00DBC3E4009B019C802212061E0071
:104290009446230063441900FFF713FC02000B004F
:1042A0000020694902F0E2FD4AE46D4B9C4200DCCB
:1042B000AAE4654B9C4201DDFFF72CFC0022624B17
:1042C00003F072FCC022674BD20504000D0003F01E
:1042D000F1F9654A06000F00644B2000290003F045
:1042E000E9F9002202900391614B2000290003F0BC
:1042F000E1F902000B005F485F4903F055FC220022
:104300002B0003F0D7F902000B0000205B4903F0FB
:104310004BFC2200049005912B002000290003F0A3
:10432000C9F902000B000498059903F0C3F9544A37
:104330004C4B03F0BFF902000B000298039903F005
:1043400033FC02000B0004000D003000390002F0C5
:1043500061FA002210003B0032000290039103F04A
:1043600023FC02000B002000290003F01DFC049038
:104370000591E1E5434A444B0698079903F09AF901
:10438000404A414B03F096F90600FFF79AFB002ADA
:1043900001D0FFF7A5FB1432D31A3A001A411100DD
:1043A00099408F4201D0FFF76FFB01231340022297
:1043B000D31A9B46FFF768FB304B9E4200DD4EE66A
:1043C0000023994698467AE602000B00FFF714FC9A
:1043D00080232E4CDB05089309942D4B2D4C002295
:1043E0000C930D9480242C4BE4020692079356E420
:1043F00043465B42984651E6424600F0C9FB07E758
:1044000002FCFFFF01FCFFFFFFFF0F00432EE63F12
:10441000EF39FAFE422EE63F396CA80C615C20BEF3
:10442000D0A4BE726937663EF16BD2C541BDBB3EBA
:104430002CDE25AF6A56113F93BDBE166CC1663F98
:104440003E5555555555C53F0000F03FFFCB9040B8
:1044500000346F3F59F3F8C21F6EA5010000F0BF92
:10446000FEFFEF3F4715F73F44DF5DF80BAE543ECC
:104470000000D03F555555555555D53F0000E03FFC
:10448000FE822B659C7500883CE4377E03B8E23FD2
:1044900006D0CF43EBFD4C3E0000F83FF0B556464A
:1044A0004D4644465F46754BF0B40A000D001900B6
:1044B00083B0060004002940994200D1BAE0002DE3
:1044C00000DC94E02D1500D1A3E06D4B12039C4657
:1044D0008023120B5B0365441A43EB0700D581E090
:1044E0006B109846E30F9B189B188022162100261C
:1044F000002764009203B818984202DC87181B1A40
:10450000B618E00F5B0001391B186400520800293F
:10451000F1D1002201929446802212062020914679
:1045200009E09F4241D0E10FC9180138CB1864005F
:10453000520800281ED0614651189F42F1DA8D18AA
:10454000AC46CD0FED07BA464D4539D0DB1B8C424A
:10455000BF417F42DB1B641A019901388B469344AB
:1045600059460191E10FC9185746CB18640052080B
:104570000028E0D123432BD1019B5B0841497210F5
:104580008C466244F10702D5802109060B4341465F
:1045900009058D181E002F003000390003B03CBC07
:1045A00090469946A246AB46F0BDA1420ED88D1862
:1045B000AC46CD0FED074D4548D09A460023CAE7DB
:1045C0006546002DC2DB7D1CAA46BFE73B00AAE77B
:1045D000019B01333ED0019A01239446134063446A
:1045E0005B08CBE7E30F52009A18640078E76B0092
:1045F0005B0803432F00002BCED00025002A31D1C9
:10460000E20A153D6405002AFAD080235B031A42B2
:1046100023D180200023400300E00B005200591CEE
:104620000242FAD02020401AED1A2300C3408C40E9
:104630001A434AE702002B00290003F03BF832003E
:104640002B0002F0E7F806000F00A5E76546002DF5
:10465000B3DBB8E70136002390E7012320205B425B
:104660000021E1E73B000200390003F09DFA02005F
:104670000B0002F0FBFB06000F008DE70000F07F4F
:1046800001FCFFFF0000E03FF8B556464D464446AA
:104690005F46A54BF0B44E00804689468A467608B0
:1046A0009E420CDDA14B9E4200DDA0E000D19BE0CC
:1046B0005346002B00DCE3E09D4B9E4A9FE09E4B5F
:1046C0009E4200DDB1E09D4B9E4200DC9FE0012355
:1046D0005B429B4642464B464046494602F0EAFF53
:1046E00002000B0006000F0002F0E4FF04000D00C2
:1046F000934A944B02F0DEFF934A944B02F08AF8FF
:1047000022002B0002F0D6FF914A924B02F082F871
:1047100022002B0002F0CEFF8F4A904B02F07AF875
:1047200022002B0002F0C6FF8D4A8E4B02F072F879
:1047300022002B0002F0BEFF8B4A8C4B02F06AF87D
:1047400032003B0002F0B6FF894A8A4B06000F0098
:104750002000290002F0AEFF874A884B03F024FABC
:1047600022002B0002F0A6FF854A864B03F01CFABC
:1047700022002B0002F09EFF834A844B03F014FAC0
:1047800022002B0002F096FF814A824B03F00CFAC4
:1047900022002B0002F08EFF0B005946020001316F
:1047A00000D170E059463000CC00390002F032F8F8
:1047B00042464B4602F07EFF774D784B2D191C196F
:1047C0002268636803F0F0F942464B4603F0ECF9C7
:1047D00002000B002868696803F0E6F953460A00F6
:1047E000002B48DB03000AE0002800D160E74246C6
:1047F0004B464046494602F00DF803000A001800F7
:1048000011003CBC90469946A246AB46F8BD644AAE
:10481000644B01F0FFFF0022634B01F007F9002811
:1048200000D154E743464A46E9E700F0CBF85F4B36
:1048300004000D009E4237DC5D4B9E425DDC0200B1
:104840000B0001F0E7FF0022574B03F0ADF9802386
:1048500006000F000022DB052000290001F0DAFF2E
:104860000B0002003900300002F000FB00238046FC
:1048700089469B462EE78022120603008A18BEE76F
:104880002B4B4C4ABBE73000390001F0C3FF4246D6
:104890004B4602F00FFF02000B004046494603F072
:1048A00083F903000A00AAE7434B9E421ADC002268
:1048B000424B03F079F9002206000F003F4B200025
:1048C000290002F0F7FE0022374B01F0A3FF0B0096
:1048D00002003900300002F0C9FA022380468946FE
:1048E0009B46F7E60B0002003549002002F0BEFAB5
:1048F0000323804689469B46ECE600222A4B03F0C0
:1049000053F9002206000F00274B2000290001F078
:1049100081FF0B0002003900300002F0A7FA0123EA
:10492000804689469B46D5E6FFFF0F440000F07F96
:10493000182D4454FB21F93FFFFFDB3FFFFF1F3ED3
:1049400011DA22E33AAD903FEB0D76244B7BA93F81
:10495000513DD0A0660DB13F6E204CC5CD45B73F4F
:10496000FF8300922449C23F0D5555555555D53FFB
:104970002F6C6A2C44B4A2BF9AFDDE522DDEAD3FEF
:104980006D9A74AFF2B0B33F711623FEC671BC3F8F
:10499000C4EB98999999C93F288B0000088B0000B7
:1049A0009C7500883CE4377E0000F03FFFFFF23F3B
:1049B000FFFFE53FFB21F9BFFF7F03400000F83F09
:1049C0000000F0BF49004B0819007047034B480036
:1049D0009C4640086044C00F7047C04600001080ED
:1049E0000A000300024330B50220002A00D130BD86
:1049F00080221206914216D00C4A0D4C8A180420CF
:104A0000A242F4D90B4A8A18A242F0D90A4A4900B4
:104A1000490803209142EAD9064A00209142E6D192
:104A200058425841E3E7002BE1D0EFE70000F0FFE8
:104A3000FFFFDF7F0000F07FFFFF0F0000207047C7
:104A4000002001497047C0460000F87FF0B5474696
:104A500080B4CB0F98464A4C4B005B0D1E1982B0B8
:104A600007000A00132E35DC002E57DB454B0400EF
:104A700033411F000F4007430D00002F24D05B0877
:104A80001C000C4020430027002807D0132E00D123
:104A900072E08022D202324199430A434346DE004B
:104AA000394B11009E1934687568380022002B00BC
:104AB00001F0B0FE009001910098019922002B00B6
:104AC00003F072F804000D002000290002B004BCBD
:104AD0009046F0BD332E0CDD802304000D00DB007A
:104AE0009E42F1D102000B0001F094FE04000D0083
:104AF000EAE7264C0D00A446012463446442DC40EE
:104B0000A446614604000142DED049080142C5D0F6
:104B10008027FF051F4188430743BFE74B005B0821
:104B2000034304000D00002BCED00B031B0B0343EB
:104B30005A42134380221B0B120313404A0C5204A7
:104B4000134319004346104ADB00D3181C685D6804
:104B500022002B0001F05EFE009001910098019967
:104B600022002B0003F020F842464B005B08D607DA
:104B7000334304001D00A7E780273F0689E7C046AE
:104B800001FCFFFFFFFF0F00488B0000EDFBFFFF64
:104B90004B0070B55B0D14000A00002B1AD14B00BE
:104BA0005B08034315D00022224B02F083FD224B09
:104BB0000A009C4222DB4B005B0D363B1F4DE31885
:104BC000AB4220DC002B0DDD1D4C1B0522401A439F
:104BD000110070BD1B4DAB42F0D102000B0001F083
:104BE00019FEF6E71D00353518DA174B02009C4216
:104BF0000ADC0B001548164900F032F8134A144B32
:104C000002F058FDE5E702000B001248124900F0DF
:104C100027F8104A104B02F04DFDDAE7084C363306
:104C200022401B051343190000220C4B02F042FDE9
:104C3000CFE7C04600005043B03CFFFFFE07000036
:104C4000FFFF0F80FF07000050C3000059F3F8C2B8
:104C50001F6EA5019C7500883CE4377E0000903CE7
:104C600030B54A00DB0FDB0752081A43110030BD94
:104C700003210A4802680A430260094802680A439D
:104C800002600849084A094B9B1A03DD043BC858D7
:104C9000D050FBDC00F012F8FBF76CFA2405004062
:104CA00054050040EC8C000000000020640100204E
:104CB000FEE7FEE7FEE7FEE7FEE7FEE7014A024BFE
:104CC0001A6070470024F4009C000020084A09493B
:104CD000094B10B51B688858FA22190A1B0618439D
:104CE0009200002300F0F0FE4904C00B084310BD01
:104CF0000405000000100140000A0020084B094A8A
:104D000009491B688858190A1B0610B51843074A39
:104D1000002300F0D9FE4904C00B084310BDC04673
:104D2000000A0020040500000010014040420F006E
:104D300070B5041E09D0FFF7C9FF050000F014F894
:104D4000FFF7C4FF401B8442F8D870BD0022044B1B
:104D50009A60044A13680133DBB213607047C0469F
:104D6000FC100140000A002070470000F7B5002346
:104D7000202877D83C4B8000C258042A14D006D88B
:104D8000022A0DD00ED80423012A14D069E0062A85
:104D90000ED00BD31A2A0DD002231B2A0BD060E0B1
:104DA000082308E0102306E0202304E0402302E06B
:104DB000802300E001232D4A1268082A04D9092A19
:104DC00005D00A21022404E00821002401E011009A
:104DD0000124A02501261C272548ED004651254D1C
:104DE000254E2D681B02AD003D400195234D2D68D9
:104DF00000958559AC466746214D3D401D43855180
:104E00008359C0259C46009BAD021D40FF23674689
:104E10001B023B402B43019D1D43009B5F01602310
:104E20001F402B003B431C4301238451154C03605E
:104E300063680F48002BFBD00024124B01255C60F7
:104E4000A123DB00C3584560A025ED0044511BB2EF
:104E5000914207D002D98A1AD34003E0521A9340F4
:104E600000E000231800FEBD788A0000A8000020A2
:104E700000700040A400002004050000A0000020F5
:104E8000FF00FFFFFC7000401E4BF0B5596C18008E
:104E90001D4A002914D0A025A12600230124ED05D8
:104EA000F600D1584F1C06D0D7187F68002F02D0CB
:104EB00027008F40AF5114333C2BF2D100234364C1
:104EC000131DA02540329446002001240F4EED050D
:104ED000DA680F49920057180A495218526C002A92
:104EE0000CD01A1F1268511C05D01968FF2902D076
:104EF00021009140A9513A00FC32506414339C4582
:104F0000E6D1F0BDFC900040AC0000200C05000094
:104F10000090004000B5202816D80C4A83009B580A
:104F2000032911D8A0220800C133FF33D2059B000A
:104F300000F0C8FB02080406002104E00C2102E096
:104F4000042100E00321D15000BDC046788A000052
:104F500020280DD8074B8000C25801239340A0227F
:104F6000D205002901D1044901E0A121C900535013
:104F70007047C046788A00000C050000030000203E
:104F8000202B0AD8A222A021D200C9058858034AA2
:104F90009B009B58D840012318407047788A000036
:104FA000F7B506000D000C008B180193019B671BE1
:104FB0009C4207D0336821781B6830009847013441
:104FC0000028F3D13800FEBD70B505000C00081EA6
:104FD00007D003F081FC2B6802005B6821002800E9
:104FE000984770BD10B5FFF7EFFF10BD10B503680F
:104FF0001B68984710BD000010B50249FFF7E4FF99
:1050000010BDC046588B000070B50500FFF7DCFFEF
:1050100004002800FFF7F0FF001970BDF0B516007E
:1050200000228DB002AB053301900D00DA77012E1E
:1050300000D80A260BAC2800310000F0DDFB0F0081
:10504000CBB228003100009300F050FBFBB23733A5
:105050000500013CDBB2092F02D8009B3033DBB2E4
:105060002370002DE7D121000198FFF7ADFF0DB0AF
:10507000F0BD10B5002A04D10368C9B21B68984777
:1050800002E0D2B2FFF7CAFF10BD10B5FFF7F1FF83
:1050900010BD70B50500FFF7ECFF04002800FFF716
:1050A000ABFF001970BD70B50500FFF7E2FF04000B
:1050B0002800FFF7A1FF001970BDF8B506000C002D
:1050C000151E04D10368C9B21B68984714E0D2B218
:1050D0000A2D0DD12A0000290ADA2D21FFF786FFBB
:1050E000614207002A003000FFF798FF381803E0FC
:1050F00021003000FFF792FFF8BD10B5FFF7DDFF8C
:1051000010BD0000F0B51E0085B00AAB1B78310061
:105110000500100017000293FFF762FC45490028C4
:1051200006D038003100FFF75BFC012804D142496A
:105130002800FFF749FF7BE0E022404B12063800D1
:10514000310000F073FC002801D03D49F0E7E02277
:105150003C4B12063800310000F054FC0028F4D11A
:10516000002200233800310000F04CFC002808D059
:105170002D212800FFF73AFF80231B060190F61827
:1051800000E00190002400202F49029BA34206D09A
:1051900000222E4B013401F069FEE4B2F5E7330042
:1051A0003A0001F037FB0F00060000F0D1FC0A22A4
:1051B000039001002800FFF731FF019BC418029BF8
:1051C0002000002B34D0039803F0BAF80B00020043
:1051D0003900300002F0E8FC06000F0028001C49EE
:1051E000FFF7F2FE2318029C0193184B00223000B7
:1051F000390002F05FFA0F00060003F029F80A22D6
:10520000010002902800FFF758FF019B013C1B188A
:105210000298019303F052F802000B0030003900AD
:1052200002F0C2FCE4B206000F00002CDDD10198B0
:1052300005B0F0BD5B8B00005F8B0000FFFFEF410E
:10524000638B0000FFFFEFC10000E03F000024403F
:10525000678B000037B51D00069BDBB200932B0067
:10526000FFF750FF3EBD10B540220021040003F0BF
:1052700012FA002320002364636410BD3F23026CF4
:1052800010B5541C2340446C9C4201D081540364EB
:1052900010BD0023036443647047436C026C934267
:1052A00006D03F21C25C01330B404364100001E093
:1052B000012040427047036C406C181A00D5403002
:1052C0007047436C026C934201D0C05C01E0012046
:1052D00040427047036C406C5A1C3F231340181A1D
:1052E00042424241D0B270470120704710B5036876
:1052F0001322DB69984710BD704700000369054A17
:105300009950FC331A6A002AFCD0002201201A624C
:105310007047C0461C050000030010B55C331A78C6
:105320001F2313400122110099400D4B0424D9671B
:10533000C221036989005C505A60DA60A022002112
:10534000D20099500122074952425A50064914305E
:105350005A500C395A5008315A50FFF79AFF10BD75
:1053600004E100E00C0500001405000010B5143045
:10537000FFF7A1FF10BD10B51430FFF7A2FF10BD5D
:1053800010B51430FFF789FF10BD0000030070B5A1
:105390005E331C780269604BD45003005D331C7887
:1053A0005E4BD450030061331C785D4B012C0CD153
:1053B00005005F352E78A225ED00565105006035B9
:1053C0002E78A125ED00565100E00024D4509623FC
:1053D000DB00994238D996231B01994237D996238D
:1053E0005B01994236D996239B01994234D9E12336
:1053F0009B01994232D99623DB01994231D9E123AD
:10540000DB0199422FD996231B0299422DD9E12322
:105410001B0299422BD996235B02994229D9E12399
:105420005B02994227D9E1239B02994225D93D4B42
:10543000994224D9E123DB02994223D9E1231B03BA
:10544000994221D8384B21E09E23DB021EE09D23A8
:105450001B031BE0354B19E0354B17E0EC239B0396
:1054600014E0344B12E0344B10E0344B0EE0344B7C
:105470000CE0344B0AE0344B08E0344B06E0802368
:10548000DB0403E0324B01E080235B05314900245B
:1054900053500423243953501100FC31CC600C626A
:1054A000C1210134890014605C309460535003784A
:1054B0001F202200D9B20840824080342648FF34A1
:1054C0005BB20251002B13DA0F230B40083B234C35
:1054D0009B089B001B1903242140A140FC348C40F5
:1054E000DD69A543C0248C4021002943D96111E026
:1054F000194C9B089B001B1903242140A140C02587
:10550000FC348C40AD005E59A643C0248C40210081
:1055100031435951026070BD0C05000014050000B4
:105520006C05000090D0030000D0BE0E00B0130048
:105530000050270000A04E0000F0750000509D00B4
:1055400000F0EB0000903A0100E0D70100B0AF039B
:1055500000705F072405000000E100E000ED00E0BE
:10556000F7B5009308AB1B7800250193FA230400DC
:105570009B0083600E4B45600833036014300F00BE
:105580001600FFF770FE23005C3327611E70009B3E
:10559000084A9B00995823005D331970019B200035
:1055A0009B009A5823005E33DD701A70FEBDC04622
:1055B0006C8B0000788A0000036910B51A00FC3279
:1055C000D2680400002A0AD0A322D20099581430CD
:1055D000C9B2FFF753FE00222369FC33DA6010BD25
:1055E00010B50248FFF7E8FF10BDC046040A0020CE
:1055F000162307B5022200930249013B0248FFF738
:10560000AFFF07BD00200040040A002010B50028AD
:1056100001D003F0E5F810BD002110B5041E8C4246
:1056200004D003F00BF9210000F0D0F9080010BD00
:105630007047000010B500F011F8FFF7F9FF0120E6
:10564000FFF776FBFDF79CF8FDF7D6F8024B002B31
:10565000FAD000E000BFF7E700000000C421114AC3
:1056600089005058104B0340C020000203435350A0
:10567000802391399B02FF39535013608023A3226A
:105680000021DB05D20099500122A1209A60074B2E
:10569000C0001950C120023180001950403019500B
:1056A0001A60704700E100E0FF00FFFF00100140BA
:1056B00002B4714649084900095649008E4402BCAB
:1056C0007047C04602B4714649084900095C490068
:1056D0008E4402BC7047C04603B47146490840007E
:1056E0004900095A49008E4403BC70470022430810
:1056F0008B4274D303098B425FD3030A8B4244D39A
:10570000030B8B4228D3030C8B420DD3FF220902DB
:1057100012BA030C8B4202D31212090265D0030B9A
:105720008B4219D300E0090AC30B8B4201D3CB0390
:10573000C01A5241830B8B4201D38B03C01A5241D2
:10574000430B8B4201D34B03C01A5241030B8B42D4
:1057500001D30B03C01A5241C30A8B4201D3CB02BF
:10576000C01A5241830A8B4201D38B02C01A5241A4
:10577000430A8B4201D34B02C01A5241030A8B42A7
:1057800001D30B02C01A5241CDD2C3098B4201D3BF
:10579000CB01C01A524183098B4201D38B01C01A3D
:1057A000524143098B4201D34B01C01A52410309B4
:1057B0008B4201D30B01C01A5241C3088B4201D363
:1057C000CB00C01A524183088B4201D38B00C01A10
:1057D000524143088B4201D34B00C01A5241411A37
:1057E00000D20146524110467047FFE701B5002044
:1057F00000F0F0F802BDC0460029F7D076E7704708
:1058000003460B437FD4002243088B4274D3030921
:105810008B425FD3030A8B4244D3030B8B4228D3C2
:10582000030C8B420DD3FF22090212BA030C8B42E8
:1058300002D31212090265D0030B8B4219D300E088
:10584000090AC30B8B4201D3CB03C01A5241830B0D
:105850008B4201D38B03C01A5241430B8B4201D3BD
:105860004B03C01A5241030B8B4201D30B03C01AE6
:105870005241C30A8B4201D3CB02C01A5241830A60
:105880008B4201D38B02C01A5241430A8B4201D38F
:105890004B02C01A5241030A8B4201D30B02C01AB9
:1058A0005241CDD2C3098B4201D3CB01C01A524120
:1058B00083098B4201D38B01C01A524143098B42A9
:1058C00001D34B01C01A524103098B4201D30B0192
:1058D000C01A5241C3088B4201D3CB00C01A5241B7
:1058E00083088B4201D38B00C01A524143088B427C
:1058F00001D34B00C01A5241411A00D20146524115
:10590000104670475DE0CA0F00D04942031000D333
:105910004042534000229C4603098B422DD3030A88
:105920008B4212D3FC22890112BA030A8B420CD398
:10593000890192118B4208D3890192118B4204D3C1
:1059400089013AD0921100E08909C3098B4201D341
:10595000CB01C01A524183098B4201D38B01C01A7B
:10596000524143098B4201D34B01C01A52410309F2
:105970008B4201D30B01C01A5241C3088B4201D3A1
:10598000CB00C01A524183088B4201D38B00C01A4E
:105990005241D9D243088B4201D34B00C01A524125
:1059A000411A00D20146634652415B10104601D3B2
:1059B0004042002B00D54942704763465B1000D33C
:1059C000404201B5002000F005F802BD0029F8D0E2
:1059D00016E770477047C0468446101C62468C46E6
:1059E000191C634600E0C0461FB501F0F9FD002810
:1059F00001D40021C8421FBD10B501F04DFD404249
:105A0000013010BD10B501F0EBFD002801DB0020D6
:105A100010BD012010BDC04610B501F0E1FD002809
:105A200001DD002010BD012010BDC04610B501F001
:105A300073FD002801DC002010BD012010BDC04610
:105A400010B501F069FD002801DA002010BD012029
:105A500010BDC0468446081C6146FFE71FB500F034
:105A600091FB002801D40021C8421FBD10B500F0F1
:105A70001DFB4042013010BD10B500F083FB002833
:105A800001DB002010BD012010BDC04610B500F0A4
:105A900079FB002801DD002010BD012010BDC046AB
:105AA00010B500F02BFB002801DC002010BD012008
:105AB00010BDC04610B500F021FB002801DA00201F
:105AC00010BD012010BDC046F0B54F464646C0B4DB
:105AD0001604360C9946330005042C0C070C150CE3
:105AE00063437E436F4365431C0CAD1964199C46A8
:105AF000A64203D980235B02984647446346250C9F
:105B0000EF191D044B464A4343432D0C24046419EA
:105B10009918C91920000CBC90469946F0BDC046A2
:105B20009E2110B5C905041CFFF7C4FF002803D14E
:105B3000201C00F005FE10BD9E21201CC90500F0B0
:105B400079FC00F0FDFD80231B069C466044F2E7D3
:105B500070B500220C4B04000D00FFF771FF002808
:105B600004D12000290002F073FB70BD064B002217
:105B70002000290002F018F802F06AFB80231B06BF
:105B80009C466044F1E7C0460000E041F8B54A0297
:105B9000430244004E00C50F240E28009B09360E18
:105BA000C90F92098D4259D0A01B002800DC8DE05E
:105BB000002E1AD1002A00D079E05A0704D00F2213
:105BC0001A40042A00D004335A0138D50134FF2C7E
:105BD00000D189E028009B015B0AE4B25B02E40586
:105BE0005B0A2343C0071843F8BDFF2CE5D0802192
:105BF000C9040A431B2800DD89E016002021C640A5
:105C0000081A8240511E8A4132439B1A5A0114D508
:105C10009B019E09300002F0ABFC053886408442AF
:105C200065DC041B330020200134E340041BA64044
:105C3000721E964100243343BFE75A07BFD1DF08E5
:105C40002800FF2C2FD1002F00D187E08022D20323
:105C500013003B435B025B0AFF24BFE7A11B002943
:105C600049DD002E29D0FF2CA7D08026F604324330
:105C70001B2900DD8DE017002026CF40711A8A40D5
:105C8000511E8A413A439B185A01D6D50134FF2C44
:105C900064D0012276491A405B080B4013438CE71D
:105CA000031ECAD100207B025B0AE4B296E70138EA
:105CB0000028AAD0FF2C9DD17FE7002A00D17CE7E5
:105CC00001390029DFD0FF2CD2D176E7002820D17E
:105CD000601CC0B2012853DD80279E1AFF043740A4
:105CE0002FD0D61A0D0095E72800002376E7614BE8
:105CF000241A334061E700294DD1611CCEB2012E38
:105D00002FDDFF292AD09B185B080C0055E70122E4
:105D10007BE7002C1BD1002B5BD0C04300280CD0AC
:105D2000FF2E7ED01B2800DD92E01D002024C54000
:105D3000201A8340581E83412B43D31A34000D0090
:105D400064E7002E00D065E700200024ABE7FF2EBB
:105D500067D08024E40440422343E3E7FF24002388
:105D60003CE7002C61D1002B7ED0002A00D124E733
:105D70009B185A0100D460E73E4A0C0013401CE710
:105D8000002C1ED1002B2FD1002A66D013000D004D
:105D900013E7012277E7002C1FD1002B5AD0C9430B
:105DA00000290BD0FF2E50D01B295FDC1F002024C0
:105DB000CF40611A8B40591E8B413B439B183400E6
:105DC00062E7002B1CD1002A4AD013000D00FF24EB
:105DD000F3E6130034000D00EFE6FF2E35D08024EB
:105DE000E40449422343DFE7002A00D1E5E68027A7
:105DF000981AFF04074000D152E7D31A0D00DCE6E1
:105E0000FF24002A00D1D8E68020DB08C00303422B
:105E100004D0D208024201D113000D00DB00FF24A0
:105E2000CBE61300FF240D00C7E6002B0DD0FF24A6
:105E3000002A00D1C1E68021DB08C9030B42EDD066
:105E4000D2080A42EAD11300E8E71300FF24B4E6BF
:105E5000012372E713003400AFE60027002022E799
:105E600080270020FF03F1E61300A6E60123A5E743
:105E7000FFFFFF7DFFFFFFFBF0B5564644465F4640
:105E80004D46F0B444024600C70F83B08846650A09
:105E9000360EBA463DD0FF2E22D00023EC008025DE
:105EA00099469B46ED0425437F3E43465C025800DD
:105EB000DB0F640A000E984636D0FF2830D08023CE
:105EC0000021E400DB041C437F38301A019048466F
:105ED00042460843724E800030587A40130087468D
:105EE000002D44D108239946063B9B46DDE701225D
:105EF000FF2000241A406402C305640AD2071C4331
:105F00001443200003B03CBC90469946A246AB46E1
:105F1000F0BD002D20D104239946033B9B46C4E7E6
:105F2000002C17D1022102E0002C0AD10121321AE3
:105F300001924A4643460A435A48920082587B409F
:105F40009746200002F014FB431F76309C404042ED
:105F50000021BAE70321B8E7280002F009FB431F3C
:105F60009D4000237630464299469B469DE70C2390
:105F70009946093B9B4698E780240022E403FF20D2
:105F8000B9E70024C2468B465A465346022AAED091
:105F9000032A7DD0012A31D1012200201A40002499
:105FA000A9E70122101A1B2856DD1A400020002400
:105FB000A1E78023DB031D424BD18023DB032B436E
:105FC0005C02640A3A00FF2095E76D01600185429A
:105FD00030D2019A0024013A01921B2201272900A4
:105FE00064006D00002901DBA84201D82D1A3C4352
:105FF000013A002AF3D16A1E95412C4301987F3063
:106000000028CEDD620704D00F222240042A00D0EF
:106010000434220103D5244A019814408030FE281C
:1060200000DD64E70122A401640AC0B21A4062E7FD
:106030002C00A9E72D1A1A220124CFE76B02BCD548
:1060400000248023DB031C436402640A4246FF20D1
:1060500051E71C42B3D1F4E721002022C140101ABD
:106060008440621E94410C43620704D00F222240F8
:10607000042A00D00434620104D5012201201A4010
:10608000002438E70122A401640A1A40002032E704
:106090008023DB031C436402640A5246FF202AE784
:1060A0009C8B0000DC8B0000FFFFFFF7430270B504
:1060B00042004C005D0AC30F4802120E460A240E2D
:1060C000C90FFF2A0FD0FF2C11D00120A24200D00F
:1060D00070BDB542FCD18B420DD0002AF8D128000A
:1060E000431E9841F4E70120002DF1D1EBE7012098
:1060F000002EEDD1E9E70020EAE7C0464302F0B503
:1061000042005D0AC30F4802440A4800120E000E06
:10611000C90FFF2A1FD0FF2822D0002A09D16E42C2
:106120006E4100280FD1002C0DD10020002D09D088
:1061300005E0002801D1002C01D08B4213D0584239
:1061400001231843F0BD002EF7D048424141012001
:1061500049420843F6E7002DDDD002204042F1E736
:10616000002CDAD0F9E78242E9DC04DBA542E6D86C
:106170000020A542E6D25842434101205B42184329
:10618000E0E7C0464302F0B542004C005E0AC30F90
:106190004802120E450A240EC90FFF2A17D0FF2C01
:1061A00019D0002A0BD170427041002C17D0002862
:1061B00007D048424141012049420843F0BD002C2C
:1061C00013D08B4214D0584201231843F6E7022023
:1061D000002EF3D1E3E70220002DEFD1E1E7002DFF
:1061E000E5D10020002EE9D0EDE7002DE9D1EAE766
:1061F000A242E8DC04DBAE42E5D80020AE42DDD2AC
:106200005842434101205B421843D7E7F0B5574657
:106210004E4645464300E0B446028846760A1F0EC5
:10622000C40F002F47D0FF2F25D0002380259A468A
:106230009946F600ED042E437F3F434642465D02F9
:10624000D20F5B006D0A1B0E904640D0FF2B39D059
:1062500080220020ED00D20415437F3BFB1842460C
:106260005746591C62408C4607430F2F5CD86F4934
:10627000BF00C9598F46002E45D108239A46063BD8
:106280009946DAE7424602282DD0032800D1C3E020
:10629000012800D0A2E0002500260240D4B27602F8
:1062A000ED05760A2E43E407264330001CBC9046D9
:1062B0009946A246F0BD002E1AD104239A46033B0C
:1062C0009946BAE72A00511E8A41901CC6E7012070
:1062D000002DC3D0280002F04BF9431F76309D40BB
:1062E00043420020BAE70124FF2514400026D6E7E8
:1062F000300002F03DF9431F9E40002376304742B4
:106300009A46994699E70C239A46093B994694E7A1
:1063100080260024F603FF25C1E735004846B2E792
:10632000350022004846AEE72904090C0800370C66
:106330003604360C2C0C7943704367437443060CC7
:1063400064183619B14203D980214902884647446E
:106350000004000C310409188D01681E8541890E66
:106360002943350CED19AD010D43290104D5012355
:1063700069081D4063460D4319007F31002925DD62
:10638000680704D00F202840042800D004352801D5
:1063900003D5274980330D401900FE29A3DC0124D1
:1063A000AD016E0A1440CDB279E78020C0030642E9
:1063B00007D0054205D128434602760A4446FF2508
:1063C0006DE706437602760AFF2568E70124611A25
:1063D0001B2905DD14400025002660E76346CBE756
:1063E0002E002023CE40591A8D406B1E9D412E4316
:1063F000730704D00F233340042B00D004367301FD
:1064000004D5012401251440002648E70124B601E3
:10641000760A1440002542E780260124F6032E4325
:106420007602760A1440FF2539E7C0461C8C00002E
:10643000FFFFFFF7F8B54A024E0043024400240E66
:10644000C50F9B09360EC90F9209FF2E00D183E0BC
:1064500001204140A01BA9425CD0002800DC95E04F
:10646000002E1CD1002A00D081E05A0704D00F2250
:106470001A40042A00D004335A013BD50134FF2CC2
:1064800000D191E001209B015B0AE4B205405B0270
:10649000E4055B0AED0723432B431800F8BDFF2CEE
:1064A000E3D08021C9040A431B2800DD90E01600D8
:1064B0002021C640081A8240511E8A4132439B1A4D
:1064C0005A0115D59B019E09300002F051F805389C
:1064D000864084426CDC041B330020200134E340FE
:1064E000041BA640721E964100243343BDE70D00F5
:1064F0005A07BCD1DF0801231D40FF2C33D1002FE8
:1065000000D190E08022D20313003B435B025B0A80
:10651000FF24BCE700284FDD002E2ED0FF2CA4D096
:106520008025ED042A431B2800DD97E01600202576
:10653000C640281A8240501E824132439B185A019D
:10654000D5D50134FF2C6DD001227B481A405B0861
:10655000034013430D0088E7002A00D07AE777E76D
:10656000031EC5D100257B025B0AE4B28FE7013828
:106570000028A4D0FF2C97D177E7002A00D174E738
:1065800001380028DAD0FF2CCDD16EE7002821D1C8
:10659000601CC0B2012858DD80279E1AFF043740D6
:1065A0002FD0D61A0D008FE701231D4000236EE780
:1065B000624B241A334058E7002851D1601CC6B200
:1065C000012E33DDFF282DD09B185B0804004CE71B
:1065D000012274E7002C1AD0FF2E1FD08024E4047F
:1065E000404223431B2800DD96E01D002024C540C7
:1065F000201A8340581E83412B43D31A34000D00C8
:106600005EE7002E00D05FE700250024ABE7002BFB
:1066100044D0C0430028F0D0FF2EE3D11300FF2464
:106620000D0022E70D00FF24002330E7002C5DD190
:10663000002B7DD0002A00D117E79B185A0100D407
:1066400056E73E4A040013400FE7002C1ED1002BF2
:106650002FD1002A65D013000D0006E701226DE757
:10666000002C1FD1002B59D0C04300280BD0FF2E87
:106670004FD01B285EDC1D002024C540201A83401B
:10668000581E83412B439B18340058E7002B1CD124
:10669000002A49D013000D00FF24E6E61300340061
:1066A0000D00E2E6FF2E34D08024E4044042234370
:1066B000DFE7002A00D1D8E68027981AFF040740B8
:1066C00000D14DE7D31A0D00CFE6FF24002A00D1F8
:1066D000CBE68020DB08C003034204D0D20802428C
:1066E00001D113000D00DB00FF24BEE6002B10D00B
:1066F000FF24002A00D1B8E68020DB08C003034253
:1067000003D0D208024200D11300DB000D00FF24A9
:10671000ABE61300FF24A8E601236EE71300340064
:10672000A3E6002700251EE780270025FF03E9E6F2
:1067300013009AE60123A6E7FFFFFF7DFFFFFFFBA3
:106740004302590A4300C20F1B0E00207E2B0EDDB0
:106750009D2B0DDC802000040143952B0BDC962043
:10676000C31AD9400B005842002A00D118007047C4
:10677000034BD018FBE7963B99400B00F3E7C0466C
:10678000FFFFFF7F70B5002830D0C317C5185D40EC
:10679000C40F280001F0ECFE9E231B1A962B0DDC83
:1067A0009622D21A95406A02520AD8B25202C00505
:1067B000520AE40702432243100070BD992B19DCF2
:1067C0009922D21A9540124A2A40690704D00F2113
:1067D0000D40042D00D00432510103D50C4B1A405A
:1067E0009F231B1A9201520AD8B2DFE7002400202F
:1067F0000022DBE705222E00121AB921D6402A001A
:10680000C91A8A40551EAA4135001543DBE7C04628
:10681000FFFFFFFBF8B556465F464D464446F0B4D1
:106820000F00FD0FAA4609037C002E005F00450FF4
:10683000490A7F0D2943C5001803BC46400A570F7B
:10684000640DDB0F3843D2009A4500D1AAE06646BA
:10685000A61B002E00DCFFE06346002B39D10300AD
:10686000134300D0D9E06B0709D00F232B40042B32
:1068700005D02B1DAB42AD416D4249191D000B02E5
:1068800000D482E0CA4B01349C4200D1FEE00A00F1
:106890005646C84BED081A4050076405520205439E
:1068A000120B640D002112030B0D1B056405120B66
:1068B0001A436308C04CF60714401C436400640884
:1068C0003443280021003CBC90469946A246AB4682
:1068D000F8BDB74B9C42C6D080231B041843382E0A
:1068E00000DDEBE01F2E00DD1EE120239B1B9C46FC
:1068F00003006746BB40984613004746F3403B43BE
:106900006746BA40571EBA4113430200F240EB1AE1
:106910009D42B6411D008A1A7642911B0B0231D569
:106920004A02560A002E00D1B4E0300001F020FEE9
:106930000300083B1F2B00DDB5E020222900D21AFE
:10694000D1409E400A009D4032439C4200DDB1E0B0
:106950001C1B631C1F2B00DDD5E020211400280028
:10696000C91A8C40D8408D400443DA40681E8541E6
:1069700011002543002476E74146314300D134E23B
:10698000310045466B0700D06FE756464807ED08D3
:10699000C9080543864B9C4235D00A036405120B97
:1069A000640D7FE76346E31A9B46002B00DC8BE017
:1069B0006746002F3CD07E4FBC4200D153E7802772
:1069C0003F0438435B46382B00DCF7E00243501E9F
:1069D00082410020D2B253194218AB4289411D00B6
:1069E000494289180B02CDD5714B01349C4200D12C
:1069F0003DE101206F4A6B080A4028401843D50743
:106A0000054351082FE72B000B4300D1CBE1802336
:106A10001B030B431A03120B44E7013E002E6DD1FA
:106A2000AE1AB5429B41091A5B42C91A350075E797
:106A30000700174300D116E701235B429C46E3445D
:106A40005B46002B00D0E0E0AA18AA429B4109183F
:106A50005B4259181500C5E7002E75D1661C7605F6
:106A6000760D012E00DCF3E0AE1AB0464545BF417D
:106A70000E1A7F42F61B370200D48FE0551BAA4244
:106A8000B641411A76428E1B9A464BE75646002283
:106A9000002507E7280001F06BFD20300300083BCC
:106AA0001F2B00DC49E72A002838824000259C4241
:106AB00000DC4DE73F49E41A1140D4E60243501E82
:106AC0008241D3B2002222E7002B00D0F3E0631C06
:106AD0009C465B055B0D012B00DC9FE0344B9C4525
:106AE00000D1C3E0AA180918AA42804140424118C7
:106AF000CD075208154349086446B4E62C4B9C4226
:106B000000D0ECE6AFE611001F3CE1400C00202B6A
:106B100000D17FE04021CB1A9A4015436A1E95416F
:106B20000021254300242DE733000700203BDF40F0
:106B30003B00202E70D04027BE1BB0400243501EA9
:106B4000824113430022E2E6002C4FD0184CA445AA
:106B500000D1ABE08024240476422143382E00DDAE
:106B6000DFE01F2E00DD43E12027BC1BA1460C0007
:106B70004F46BC40A0462C004746F4403C434F469D
:106B8000BD406F1EBD41F1402C43151BAA429241EE
:106B9000411A5242891A64469A46BFE64146454622
:106BA000314300D0BEE6002600240025F2E6C046B0
:106BB000FF070000FFFF7FFFFFFF0F801F2B59DC47
:106BC0002027FF1ABC46070063469F405B46B94634
:106BD0001700DF40B8464F4643461F4363469A407E
:106BE000531E9A415B463A43D840F4E60C002C43CE
:106BF0005CD0F643002E55D1551BAA42A441411A40
:106C00006442091B9A46644688E6964FBC4200D00F
:106C1000D8E628E6002280E700208FE70B002B4310
:106C2000002C00D0C2E0002B00D101E1030013438F
:106C300000D118E6AB18AB42B6410918764271187C
:106C40000A0200D409E1884A1D00114064460AE6A0
:106C5000002C5BD10E002E4300D08AE001001143CE
:106C600000D1C2E0010015009A46FCE5644600210F
:106C700000258FE620235B429C46DC4463460700E8
:106C8000DF405B46BC46202B00D1ACE040235F4692
:106C9000DB1B98400243501E8241634613431A0097
:106CA000002098E66F4CA44500D057E7010015007E
:106CB00064469A46D7E5002C39D10C002C436ED09F
:106CC000DB43002B1AD0674CA44568D0382B00DD7D
:106CD000A4E01F2B00DDAEE020240F00E41AA74043
:106CE000B9462F00DF40B846A3464F4644462743E7
:106CF0005C46A5406C1EA541D9403D43AD18954268
:106D00009B4109185B42591864466BE60C002C4302
:106D100015D1010011437BD0010015009A46514C5A
:106D2000A1E50D43691E8D410021ECB22DE74D4CCC
:106D3000A44534D0802424045B422143C6E70400E8
:106D400014434ED0ED084C072C438025C9082D0371
:106D5000294208D0C6082E4205D1D2084107114366
:106D60000C009A463100620FC900E50011433D4C0A
:106D700079E50600164300D175E5AE1AB0464545E3
:106D8000BF410E1A7F42F61B370200D4F4E5551BB3
:106D9000AA42B641411A7642891B9A4663E5010030
:106DA000150064465FE5002200257BE5002B3BD003
:106DB0000300134315D0ED084B072B438025C9086A
:106DC0002D03294207D0C4082C4204D141070B00EF
:106DD0002100D2081343C9005A0F1143DD00214C92
:106DE00041E5204C3FE5002054E700260025D1E591
:106DF00034000F00203CE7403C00202E2BD04027E1
:106E0000BE1BB1400D43691E8D4100212C43BCE6E1
:106E1000802100260903134C0025BBE50D43691EA4
:106E20008D410021EDB269E7010015000D4C1AE516
:106E30000100150017E51C000F00203CE7403C0056
:106E4000202B0CD04027FB1A99400D43691E8D4121
:106E50000021254352E70021D4E71D0092E50021DF
:106E6000F3E7C046FF070000FFFF7FFFF0B556467F
:106E70004D4644465F46F0B41D000E034C00CB0F58
:106E800087B0070092468146360B640D98466AD05B
:106E90006D4B9C4235D08022430F12041343F60001
:106EA0001E43C3009946694B00279C460023644457
:106EB00002932B0368001B0BED0F51469B46400DC0
:106EC000009500D178E0604B98426CD05B46DA00C8
:106ED0004B0F802109040B4313439B465346D900B3
:106EE0005A4B9C46002360444246201A6A40924610
:106EF00001901F430F2F00D9B0E05548BF00C05983
:106F00008746374300D088E000239946023308279C
:106F100000260293CDE74346B34649460093029BC1
:106F2000009A9246022B00D0BFE100215346012275
:106F3000002689461A40444B002136030C0D2405D7
:106F4000360B2643434C1B0526401E437600D207D2
:106F5000760816434846310007B03CBC9046994637
:106F6000A246AB46F0BD330003434FD0002E00D104
:106F7000BCE1300001F0FCFA03000B3B1C2B00DDF0
:106F8000ADE11D220100D31A08393A008F408E402E
:106F9000DA40B9461643304B00279C460023604434
:106FA0004442029385E753465A4613432CD10023AB
:106FB00000219B46023397E70B4320D05B46002B12
:106FC00000D19EE1584601F0D3FA03000B3B1C2B85
:106FD00000DD8FE102005946083A91408B461D21A1
:106FE000CB1A5146D9400B0059460B4351469B469C
:106FF0009140194B9C4660444042002374E70023B3
:1070000000219B4601336FE703236DE70023994678
:1070100001330427002602934BE703230C27029336
:1070200047E70122D51A382D00DCB0E153461A405B
:1070300000210023002689467EE70023802699460A
:1070400000223603004B77E7FF07000001FCFFFF3B
:107050005C8C0000FFFF0F80F30300005E4500D949
:1070600072E100D16DE1019B4D46013B019300238C
:10707000340002935B461E020B0E1E430B02039369
:10708000330C994633041B0C494620000093FEF74D
:107090002DFB009B370043430600494620009846DD
:1070A000FEF7AAFB2C0C09040C43A04509D9E419EE
:1070B000731EA74200D95CE1A04500D859E1023E09
:1070C000E4194346E41A49462000FEF70FFB03008B
:1070D000009A80465343494620009B46FEF78CFBAE
:1070E0002A040904120C0A4393450DD94346D219C8
:1070F000013B974200D93AE1934500D837E102239A
:107100005B429C46D219E0445B46D21A43463604A1
:1071100033439B460399180C0B0C1D00059309047F
:107120005B46090C0C001B041B0C4443049159439F
:107130006B4368431B190D0CEB189C4203D9802448
:107140006402A44660441C0C09041B04090C2018AA
:107150005D18824200D2DEE000D1D7E0161A029B11
:107160009C465D1BAC459B415B42F61AB74200D181
:1071700006E149463000FEF7B9FA009B040043439C
:10718000494630009846FEF737FB2E0C09040E43A3
:10719000B04509D9F619631EB74200D9F3E0B045EE
:1071A00000D8F0E0023CF6194346F31A49461800AD
:1071B0000293FEF79BFA009B060043434946029860
:1071C0009846FEF719FB2D0409042D0C0D43A84524
:1071D00009D9ED19731EAF4200D9D6E0A84500D8F1
:1071E000D3E0023EED192404210043463143049EBE
:1071F000059A3000ED1A0B040C0C1B0C5843664327
:10720000534354439A19030C9B189E4203D980227E
:107210005202944664441A0C00041B04000C141916
:107220001B18A54250D34DD001231943964A019B08
:1072300094466344002B00DCF3E64A0709D00F2292
:107240000A40042A05D00A1D8A42894149428B44DA
:1072500011005A46D20108D55A468C4B1A40934623
:107260008022D2009446019B6344894A934200DD08
:107270005BE65A46C90850070843560251460122A8
:107280005B058146360B5B0D0A4055E680231B03E8
:107290001E4211D05A461A420ED15E461E43360394
:1072A000360B2A0089467B4B46E6032B00D1E1E0F2
:1072B000012BBBD11A40BBE61E433603360B4246B8
:1072C000744B39E6002BB1D07D194A1EAF4252D91A
:1072D0001100A542A8D1039A9A42A5D1A6E70300BE
:1072E0003E00283B9E400023994654E601F040F9B9
:1072F000203041E603005246283B9A400021934645
:1073000077E6504601F034F920305EE6029B002615
:10731000AB4200D323E7039E0299B44661448846FA
:10732000B045B6415B467642F619B218013B029170
:10733000974213D290424FD800D18EE0161A9B4646
:107340000DE7894500D28EE674084B46F6073500F6
:107350005B081D434B46DB0702938BE69742EDD15A
:107360000399029CA142E5D93E1A9B46F7E698464E
:10737000CAE61E00A5E6AC423ED874D0110053E721
:107380000121494252E71C000EE71E002BE71F2D8A
:107390003CDC20230A0058465B1B9840EA40994099
:1073A0000243481E81415E461143EE404B0709D01F
:1073B0000F230B40042B05D00B00191D99429B4154
:1073C0005B42F61833023CD55346012200211A4095
:1073D000002601238946AFE502235B429C46039CBD
:1073E000E344A446029B63449846A045B6417642D6
:1073F000F6190293B218B1E603988A1E4100814241
:10740000B6417642F619AD19039161E71F22524247
:10741000D31A5A46DA401300202D29D0402258466C
:10742000551BA8400143481E814107200B431840CB
:107430000026002809D00F2200261A401900042A2D
:10744000BBD10B0070077602360BDB08034399466D
:10745000012253461A4000236EE502998D42BBD8A3
:107460009B4600267BE603989842C5D3110032E77D
:107470000020D7E780265B4636031E433603360BD3
:10748000009A8946034B57E5FF030000FFFFFFFE0C
:10749000FE070000FF070000F0B55F4656464D4668
:1074A0004446F0B41F035C00DB0F9A46194B0E03F1
:1074B0004D00C90F8046360B6D0D8B4691463F0B34
:1074C000640D9D4219D0134B9C421BD00123A54251
:1074D00006D018003CBC90469946A246AB46F0BD8B
:1074E000BE42F6D1C845F4D1D34510D0002DF0D11D
:1074F000304303005A1E9341EBE73100012301435F
:10750000E7D1E0E73A430123002AE2D1DEE7002396
:10751000DFE7C046FF070000F0B55F464446564629
:107520004D46F0B41F033C0B2C4F0E034D00A346F9
:107530005C008446360B6D0DC90F9046640DDB0F61
:10754000BD422BD0254FBC422ED0002D0ED1304352
:107550000700814678427841002C17D15F463A43B4
:1075600014D14B460020002B0AD006E0002C02D19B
:107570005846024301D099421AD001234842184389
:107580003CBC90469946A246AB46F0BD0028F2D0DE
:1075900058425841012240421043F1E73700074367
:1075A000D0D002204042EBE75F461743CDD0F8E74A
:1075B000A542E2DC05DB5E45DFD808D000205E4551
:1075C000DED248424841012340421843D8E7C4452F
:1075D000D3D80020C445F4D3D2E7C046FF0700004B
:1075E000F0B55F464D4644465646F0B41C03240BA6
:1075F000A4462F4C0F034D005E00C90F80463F0B81
:107600006D0D8B469146760DDB0FA54220D0284CA0
:10761000A64222D0002D12D1384344424441002ECC
:1076200020D0002C0DD05C42634101245B421C43FE
:1076300020003CBC90469946A246AB46F0BD002EC9
:1076400017D05B4519D05B465C4201231C43EFE732
:10765000390002240143EBD1D9E7614602241143EA
:10766000E6D1D7E761460A43DBD100240028DFD00A
:10767000E9E761460A43E4D1E5E7B54203DD0122CB
:107680005C421443D4E7B542CDDB6745DBD809D073
:1076900000246745CCD259464C42614101244942FD
:1076A0000C43C5E7C845CED80024C845F3D3BFE78F
:1076B000FF070000F0B55F4656464D464446F0B41D
:1076C0000D0399464E002B0B87B00700924680466B
:1076D0009B46760DCC0F002E69D06D4B9E4235D067
:1076E0005B468022DD001204430F13432B439B466D
:1076F000C3009846674B00279C46002366440193CD
:107700004A4615035000D20F53462D0B400D9146AB
:1077100000D176E05E4A90426CD080225B0F12046A
:1077200013435C4AED0094461D4353460022DB00A0
:10773000604449463618701C6140029017430F2F71
:1077400000D9AFE05448BF00C759BF465B461F434E
:1077500000D088E000239B46984602330827019317
:10776000CEE74946022A6AD0032A00D109E2012A5B
:1077700000D0BBE111400022002300259046CCB28E
:1077800000212D030A0D12052D0B1543434A1B053D
:1077900015401D436D00E4076D0825434046290050
:1077A00007B03CBC90469946A246AB46F0BD0343A9
:1077B00052D05B46002B00D18AE1584600F0D8FE3B
:1077C00003000B3B1C2B00DD7BE11D22D31A3A008A
:1077D00001005D46DA4008398D4013008F402B438D
:1077E0009B46B8462E4B00279C46002360444642E9
:1077F000019385E752462A432CD10025002302221B
:1078000097E752462A4321D0002D00D154E12800A9
:1078100000F0AEFE03000B3B1C2B00DD46E11D21FA
:10782000CB1A51460200D9405346083A954093403E
:107830000D431B4A944660444042002279E70124EC
:1078400000220C40124B0025904699E700250023AA
:1078500001226EE703226CE700239B469846013322
:10786000042701934CE703230C27019348E70023E7
:107870008025984600242D03054B81E75D4643464D
:10788000019A6FE75D4643462100019A6AE7C046C8
:10789000FF07000001FCFFFF9C8C0000FFFF0F8032
:1078A000F30300004246120C91461A0C94464246DD
:1078B00017044A461B041B0C5A43604690464A462E
:1078C00042431000039262461C003F0C7A437C4303
:1078D00042440192220C9246019A5244904506D9A4
:1078E0008246802040028046C24450460390100CDD
:1078F000049048462404240C1204121905922A0C00
:107900002D042D0C68432C00824648467C4350438E
:107910008146200C8046574357444744BA4503D913
:10792000802040028046C144380C3F04B846484499
:107930002404240C01900498A04440440490584628
:10794000000C814658460404200C82460700484635
:107950005F434C464343604660436446834650461B
:107960004443380C8446E4186444A34203D980237A
:107970005B029C46E34448463F04230C3F0C24042E
:10798000E419574668436F4384464D465046554375
:107990004243380C814662444A445B44944503D9CF
:1079A000802040028446654403983F04834604983F
:1079B0003F0C8446E344C345804140428246100464
:1079C00084460198674484466744A344BC46A34563
:1079D000A4419946D44464428742BF41D445804182
:1079E000E144A04699459B417F424042C844074339
:1079F000120CBA18A045A4415F423B0064422343E5
:107A0000D71843467D19DB0D6D021D435B465A02B4
:107A1000059B1A43531E9A415B46DB0D1A434346AE
:107A20005B021343EA0107D501225C08134023439C
:107A3000EA07029E13436D08574AB218002A4BDD2D
:107A4000580709D00F201840042805D0181D984267
:107A50009B415B42ED180300E80104D54F4A1540F5
:107A60008022D200B2184E48824200DDE7E60124AF
:107A7000DB08680718436D02530580462D0B5B0D2C
:107A80000C407DE6802259461203114208D015426F
:107A900006D115432D0398462D0B4C46414B6FE6FE
:107AA0005D4615432D032D0B3E4B69E603005546FD
:107AB000283B9D400023BCE6504600F059FD203095
:107AC000A8E60300283B9F400023BB46984689E672
:107AD00000F04EFD203073E60124A61A382E07DD93
:107AE00000220C4000230025904649E6029EA3E7B1
:107AF0001F2E20DC20222C001800921BF040944006
:107B000093400443581E83411C43F540630709D04A
:107B10000F232340042B05D023001C1D9C429241BF
:107B20005242AD182B021FD5012400220C40012324
:107B30000025904624E61F202C004042821AD440A3
:107B4000202E1CD04022961BB5402B43581E83414B
:107B50000720234318400025002809D00F220025C4
:107B60001A401C00042AD8D1230068076D022D0B8F
:107B70000124DB08034398460C40002300E600255F
:107B8000E3E780220124120315432D0398462D0BB1
:107B90000C40044BF4E5C046FF030000FFFFFFFE6E
:107BA000FE070000FF070000F0B557464E46454669
:107BB000E0B40E001100F20F9246C500420F180308
:107BC00037037400400A4E0F7F0A3043CF4E1743ED
:107BD0005A00640D520DDB0FC900B24200D1E5E03E
:107BE00001267340A61AB446534500D1AFE0002EDB
:107BF00000DC0DE1002A3AD103000B4300D0E4E0A1
:107C00006B0709D00F232B40042B05D02B1DAB4253
:107C1000AD416D427F191D003B0200D488E0BB4B93
:107C200001349C4200D110E13A00B94B51461A4050
:107C300001235007ED08520264050543120B640D41
:107C40000B400021280012030D0D120B64052D05B9
:107C500015436208AF4CDB072C40144364006408F2
:107C60001C4321001CBC90469946A246F0BDA74B80
:107C70009C42C5D080231B0418436346382B00DD8B
:107C8000FDE01F2B00DD30E1624620239B1A02003D
:107C90009A40664690460A009940F24046464B1E7E
:107CA00099413243114363460200DA40691A8D421A
:107CB0009B410D00BA1A5B42D71A3B0235D57A02B6
:107CC000530A98464346002B00D1C4E0404600F0DA
:107CD0004FFC0300083B1F2B00DDC5E020222900DC
:107CE000D21A4746D1409F400A009D403A439C42E9
:107CF00000DDC0E01C1B631C1F2B00DDE4E0202125
:107D000014002800C91AD8408C408D400443DA4042
:107D1000681E854117002543002471E742466346EB
:107D20001A4300D14CE2674645466B0700D069E72D
:107D3000012351467807ED08FA080B4005437349C3
:107D40008C4238D012036405120B640D79E7002EC3
:107D500000DC9AE0002A47D06C4A944200D14FE7F9
:107D60008022120410436246382A00DC08E10143F5
:107D7000481E81410022C9B24919D219A942BF4106
:107D80000D007F42BF183A0200D442E15F4A01343D
:107D9000944200D14EE101205D4A69083A402840F2
:107DA0000843D507054357089A4629E706000E43BE
:107DB00000D017E714E72900114300D1F9E1802131
:107DC00009030A431203120B3BE701235B42984667
:107DD000C4446346002B72D1691A8D429B413F1AFD
:107DE0005B42FF1A0D0068E702000A4300D107E773
:107DF000012252429046C4446246002A00D0E6E086
:107E00006918A942B6413F187642F7190D00BAE742
:107E1000002E00D080E0621C5205520D012A00DCC9
:107E2000F9E06A1A91464D45B6413A1A7642921BDC
:107E30009046120200D499E04D1BA9428941C71B0C
:107E400049427A1A90469A463CE752460123002559
:107E500013400022F5E6280000F08AFB20300300E2
:107E6000083B1F2B00DC39E72A0028388240002518
:107E70009C4200DC3EE7264FE41A1740C0E601436F
:107E8000481E81410022C9B210E7002E00D0F1E067
:107E9000621C94465205520D012A00DCA0E01B4AE8
:107EA000944500D1C5E06918A94292413F18524259
:107EB000D2194908D5070D4357086446A0E6134B6D
:107EC0009C4200D0D9E69BE611001F3CE1400C002B
:107ED000202B00D180E04021CB1A9A4015436A1E26
:107EE00095410027254300241FE763460200203BFD
:107EF000DA406346202B71D0402366469B1B984096
:107F00000143481E814111430022CFE6FF070000D4
:107F1000FFFF7FFFFFFF0F80002C48D0CA4CA2421A
:107F200000D1A2E07442A1468024240427434C4699
:107F3000382C00DDDBE01F2C00DD44E14E46202420
:107F4000A41B3E00A640A246B0464C462E00E6408A
:107F5000B4464646644626435446A5406C1EA54199
:107F600034002C434D46EF400D1B28E04A46434663
:107F70004D461A4300D0A5E6002300240025DEE686
:107F80001F2A5ADC66462022921B06009640914624
:107F9000B04662460E00D640424616434A469140DD
:107FA0004A1E9141020060463143C240E4E63C0073
:107FB0002C435AD0F443A146002C52D14D1BA94268
:107FC0008941C71B49427F1A14009A4675E69E4AAA
:107FD000944200D0C7E613E600227FE700208FE737
:107FE000002C00D0C8E03B002B4300D10FE1030080
:107FF0000B4300D104E66918A9429B413F185B423C
:10800000DF193B0200D41AE1904B0D001F4064467B
:10801000F6E59A4689E63A002A43002C5CD1002A0C
:1080200075D102000A4300D1CAE007000D009A464C
:10803000E6E564460022002581E662460600203A15
:10804000D6406246B046202A00D1B7E040226646BC
:10805000921B904001434246481E81411143002239
:108060008AE6794CA24200D061E707000D001400B7
:108070009A46C5E5002C41D13C002C4378D0F4430E
:10808000A146002C20D0704CA24271D04C46382C16
:1080900000DDB2E01F2C00DDBCE02026341BA24630
:1080A0003C005646B4404E46A0462C00F440A44640
:1080B000444666463443A4465446A54064466E1E74
:1080C000B54125434C46E7406D188D4289413F1824
:1080D0004942CF19140056E6002A2FD102000A4364
:1080E00000D184E007000D009A46574C88E53D43D7
:1080F0006F1EBD41ECB200270D1B60E7524CA2423F
:1081000036D0744280263604A1463743BEE70200CB
:108110000A4300D174E56A1A90464545B6413A1AB9
:108120007642921B9446120200D4F7E54D1BA942F9
:108130008941C71B49427F1A9A4661E502000A43FA
:108140003AD0ED087C072C438025FA082D032A42FB
:1081500008D0C7082F4205D145072C003A009A469F
:10816000C9080C43670FD200E5001743364C47E5BA
:1081700007000D00140043E53A002A4343D00200F3
:108180000A4319D0ED087C072C438025FA082D03FB
:108190002A4207D0C6082E4204D147073C003200CD
:1081A000C9080C43D700620FE50017439A46264CD6
:1081B00026E50022002544E5234C21E5002049E77F
:1081C00000230025BBE54C463E00203CE6404C46E3
:1081D000B446202C31D040244E46A61BB7403D4328
:1081E0006C1EA54164462C4300270D1BE7E6802248
:1081F00000231203144C0025A1E53D436F1EBD4131
:108200000027EDB260E707000D000F4CF8E407000F
:108210000D00F5E44E463C00203EF440A0464C469E
:10822000202C0ED040244E46A41BA7403D436F1E79
:10823000BD4144460027254346E70027CFE70D0010
:1082400073E50027F2E7C046FF070000FFFF7FFF4E
:108250000B0330B5134D1A0B4B005B0DC90F0024F7
:10826000AB4211DD104CA34210DC80246403224396
:108270000E4CE41A1F2C0CDD0D48C31ADA40130013
:108280005C42002900D11C00200030BD094BCC18F5
:10829000FAE7E040084CA44663449A4013000343C5
:1082A000EEE7C046FE0300001D040000330400009A
:1082B00013040000FFFFFF7FEDFBFFFF70B50028F8
:1082C00030D0C317C4185C40C50F200000F050F92F
:1082D000174B184A1B1AD21A1F2A18DD164AD21A2F
:1082E0009440002224035B05240B5B0D0021100049
:1082F00024030A0D1205240B1443104A1B051440D5
:108300001C436400ED0764082C43210070BD21006C
:1083100091400A000B21081AC4405B052403240B7A
:108320005B0DE3E70025002300240022DEE7C046C2
:108330001E0400003304000013040000FFFF0F8040
:1083400070B5051E28D000F013F9154B154A1B1AFD
:10835000D21A1F2A16DD2C00134A0025D21A944087
:108360005A052403240B520D002124030B0D240B6A
:108370001B0523430D4C1205234013435B002800CB
:10838000590870BD0B212C00081AC44095402403E5
:108390005A05240B520DE7E700220024E4E7C0460B
:1083A0001E0400003304000013040000FFFF0F80D0
:1083B0004200120E511C4302C9B270B55D0AC40FCF
:1083C000012915DDE02189008C466D071B0B6244F5
:1083D000002128000D0D2D052B431C4D52052B406F
:1083E000520813435B00E4075B082343190070BD88
:1083F000002A15D1002D1FD0280000F0B9F80A2856
:108400001DDC0B232A001B1ADA4013000200153270
:1084100095400F4A1B03121A52051B0B520DD7E74A
:10842000002D06D080221B0B120313436D07094A4F
:10843000CEE7084A0023CBE700220023C8E7030069
:108440000B3B9D402B000025E3E7C046FFFF0F805C
:1084500089030000FF0700004B0070B55E0D0C03A0
:10846000751C640A420F6D052243C90FC4006D0DCF
:10847000012D2ADD3B4BF318FE2B1ADC002B42DDCD
:108480008001451EA841D2001043620F02435007ED
:1084900004D00F201040042800D004328020C004F3
:1084A000104021D00133FF2B03D09201520ADBB2DE
:1084B00001E0FF2300225202520ADB0513435B0056
:1084C000C9075B080B43180070BD002E07D014438A
:1084D000EFD08020D20080040243FF23D7E722435D
:1084E0000023002A03D00522D208FF2B03D052021A
:1084F000520ADBB2DFE7002A32D08020C0030243F9
:108500005202520AD7E71800173014DB802000040B
:1085100002431E20C01A1F280FDC2500124BF3183F
:108520009D406E1EB5419A402B0013432200C2406D
:108530001A430023ABE70023D5E702256D42EB1A6F
:108540001500DD40202809D0084BF3189A40144349
:10855000621E9441220000232A4398E70022F6E796
:108560000022A8E780FCFFFF82FCFFFFA2FCFFFFC8
:108570001C2101231B04984201D3000C10391B0A53
:10858000984201D3000A08391B09984201D3000917
:10859000043902A2105C40187047C046040302026E
:1085A0000101010100000000000000000B0010B5F7
:1085B0000100180000F002F810BD000070B5054C75
:1085C00005001300201E04D00A000220290000E04C
:1085D00000BF70BD00000000014B18687047C04626
:1085E00048010020084B10B50400002B02D00021E8
:1085F00000E000BF054B1868836A002B00D0984745
:10860000200000F07FF9C04600000000DC8C000074
:108610000E4B70B500251E000D4CE41AA410A542A7
:1086200004D0AB00F35898470135F8E700F06CF937
:10863000084B00251E00084CE41AA410A54204D0E3
:10864000AB00F35898470135F8E770BD4C010020A6
:108650004C0100204C0100205C01002010B5034BB0
:108660000100186800F066F810BDC04648010020FF
:1086700010B5034B0100186800F016F810BDC04695
:1086800048010020002310B59A4203D0CC5CC454AA
:108690000133F9E710BD03008218934202D019702C
:1086A0000133FAE77047000030B500293ED00439A5
:1086B0000B68002B00DAC9181D4A13681400002B40
:1086C00002D14B60116031E08B420DD90A688818E5
:1086D000834203D118685B6882180A604B6021608E
:1086E00024E08A4203D813005A68002AF9D11D6891
:1086F0005C198C420BD109686918581819608242BC
:1087000014D110685268411819605A600EE08C420A
:1087100002D90C23036009E008680C18A24203D1B7
:1087200014685268201808604A60596030BDC0461D
:108730006C0A0020032370B5CD1C9D43083506004C
:108740000C2D01D20C2505E0002D03DA0C230020AE
:10875000336040E0A942F9D81F4B1C681A00210081
:10876000002913D00B685B1B0DD40B2B02D90B60B7
:10877000CC181EE08C4202D1636813601AE04B688B
:1087800063600C0016E00C004968E9E7134C2368AD
:10879000002B03D1300000F08DF82060290030005C
:1087A00000F088F8431CD1D00323C41C9C43A04292
:1087B0000AD12560200007220B30231D9043C31AE5
:1087C00009D05A42E25006E0211A300000F072F857
:1087D000431CEED1BAE770BD6C0A0020680A002085
:1087E000104B70B51C680500A36B002B15D1182029
:1087F000FFF734FF0C4BA06303800C4B0122438036
:108800000B4B83800B4BC3800B4B038105234381B0
:10881000063383810023026143610022A36B1D6143
:108820005A6170BD480100200E330000CDABFFFF40
:10883000341200006DE6FFFFECDEFFFF154B10B5B4
:108840001C68A36B002B15D11820FFF707FF124BF4
:10885000A0630380114B01224380114B8380114B95
:10886000C380114B03810523438106338381002399
:1088700002614361A46B0D4A206961690C4BFDF7ED
:1088800023F90122002380185941206161614800C9
:10889000400810BD480100200E330000CDABFFFFA3
:1088A000341200006DE6FFFFECDEFFFF2D7F954CDC
:1088B0002DF45158002370B5064C050008002360C4
:1088C00000F012F8431C03D12368002B00D02B606A
:1088D00070BDC046740A00200023C25C0133002A28
:1088E000FBD1581E70470000044A1368002B03D0C8
:1088F0001818106018007047014BF9E7700A002043
:10890000780A0020FEE7C046F8B5C046F8BC08BCAF
:108910009E467047F8B5C046F8BC08BC9E467047F6
:10892000303238343635373039313333353530300D
:1089300030303030304142434420343631333235E8
:10894000373938304142434420000003010100041C
:1089500001020003020402050206020702010108E7
:1089600000020108020001070006000500040003E0
:10897000000202060100020501010200000083005E
:108980009300A500AF00C400DC00F700060126013B
:108990000303000F0B0D0B070E070D0B0F03080F42
:1089A0000B0B0C0F000103070F1F1E1C18100707ED
:1089B000081F171D151F1E071D171F07101F1B1B44
:1089C0001C1F2A302344373839433435364231327C
:1089D000334170726F6772616D2073697A653A0016
:1089E00020320020380020302000392030004E6F27
:1089F0002C2049442C207420286D73292C2064617C
:108A00007461582C2064617461592C206461746114
:108A10005A2C20706572696F6420286D7329002CB0
:108A20002020002C202C200020202000535F41001B
:108A3000535F4200534E52004D414700425249009D
:108A400041434300544D5000505F3000505F3100AF
:108A5000505F3200434E5400000000000000000050
:108A6000932F0000592F00007F2F0000892F000056
:108A7000B92F00007D2F000003000000020000005D
:108A800001000000040000000500000011000000CB
:108A90000C0000000B000000120000000A000000A3
:108AA000060000001A00000014000000170000007B
:108AB000160000001500000010000000FFFFFFFF7F
:108AC000FFFFFFFF000000001E0000001900000073
:108AD0001800000007000000080000000900000066
:108AE0000D0000000E0000000F0000001C00000040
:108AF0001B0000001D00000013000000706F7700D5
:108B00007371727400000000E2652F227F2B7A3CA3
:108B1000075C143326A6813CBDCBF07A8807703CF5
:108B2000075C143326A6913C4FBB610567ACDD3F63
:108B3000182D4454FB21E93F9BF681D20B73EF3F84
:108B4000182D4454FB21F93F000000000000304381
:108B500000000000000030C30D0A006E616E006965
:108B60006E66006F7666002E0000000000000000B8
:108B700000000000FD520000A14F00006D530000F6
:108B80008153000077530000F9520000ED520000BD
:108B90008D53000019530000E9520000CA5F000025
:108BA000EE5E0000AC5F0000845F0000AC5F000080
:108BB000785F0000AC5F0000845F0000EE5E0000A4
:108BC000EE5E0000785F0000845F0000306000000F
:108BD0003060000030600000B25F0000EE5E000018
:108BE000EE5E0000985F0000825F0000985F00006A
:108BF000785F0000985F0000825F0000EE5E00007A
:108C0000EE5E0000785F0000825F000030600000D0
:108C100030600000306000003C600000286300000D
:108C20008662000086620000846200001A63000011
:108C30001A63000010630000846200001A630000E1
:108C4000106300001A6300008462000020630000CB
:108C50002063000020630000AA6300005C70000035
:108C60002A6F000030700000206F0000307000009C
:108C70003A70000030700000206F00002A6F000082
:108C80002A6F00003A700000206F0000166F00008D
:108C9000166F0000166F00008C720000A4780000B0
:108CA0006477000064770000627700007C78000041
:108CB0007C7800006E780000627700007C7800000D
:108CC0006E7800007C7800006277000084780000F5
:108CD0008478000084780000847A0000E800002096
:048CE0000000000090
:088CE4009074FF7F0100000005
:108CEC000000000001000000288A00002C8A00000F
:108CFC00308A0000348A0000348A0000388A000070
:108D0C003C8A0000348A0000348A0000408A00004B
:108D1C00448A0000488A00004C8A0000508A0000F7
:108D2C00548A0000288A00000000008000000080A7
:108D3C000000008040400000404040004040404067
:108D4C004040409A9A9A0000F6FF00000A00FFFF8C
:108D5C00010000000A00FFFF0A00FFFF1A1B1C00A5
:108D6C00F6FF0000FD02000003040A17181909079A
:108D7C0006000000F6FF0000010000000024F400D3
:108D8C0003000000020000000A000000FFFFFFFFCC
:108D9C0000000000010000000000020001000000C3
:108DAC00FFFFFFFF000000000200000000000400B5
:108DBC0002000000FFFFFFFF0000000003000000A6
:108DCC00000008000300000000000000000000008C
:108DDC000000000000000000000000000000000087
:108DEC000000000000000000428A000000000000AB
:108DFC000000000000000000000000000000000067
:108E0C000000000000000000000000000000000056
:108E1C000000000000000000000000000000000046
:108E2C000000000000000000E800002039010000F4
:108E3C00C51500001D320000F15500000D010000A9
:048E4C000000000022
:0400000300004C713C
:00000001FF
